S01E00004652444D5F4B4C34335A5F4F4C323338355F44656D6F2E7372656376
S113000000600020E9040000350500003905000007
S113001000000000000000000000000000000000DC
S11300200000000000000000000000003D0500008A
S1130030000000000000000041050000450500002C
S1130040490500004D05000051050000550500005C
S113005031050000310500003105000031050000C4
S1130060590500005D0500006105000065050000FC
S1130070690500006D0500007105000031050000F0
S11300803105000031050000310500003105000094
S11300903105000031050000310500007505000040
S11300A03105000031050000310500003105000074
S11300B0B5510000310500005151000015510000F8
S1130400FFFFFFFFFFFFFFFFFFFFFFFFFE3FFFFFB9
S113041010B5064C2378002B07D1054B002B02D0D6
S1130420044800E000BF0123237010BD70E0FF1FEB
S113043000000000B4C0000008B5084B002B03D036
S11304400748084900E000BF07480368002B03D0B1
S1130450064B002B00D0984708BDC04600000000A2
S1130460B4C0000074E0FF1F6CE0FF1F0000000038
S1130470164B002B00D1144B9D46402292029A1A2F
S1130480924600218B460F461348144A121A09F06B
S11304906EFD0F4B002B00D098470E4B002B00D065
S11304A098470020002104000D000D48002802D0C8
S11304B00C4800E000BF09F02BFD2000290005F0E6
S11304C0AFFC09F00FFDC0460000080000600020EA
S11304D0000000000000000070E0FF1F1CE1FF1F8F
S11304E0000000000000000072B60A480A490160DA
S11304F00A6882F30888094880470949094A0A4B6F
S11305009B1A03DD043BC858D050FBDC62B6074895
S11305108047000008ED00E000000000B19B0000EF
S1130520DCC0000000E0FF1F70E0FF1F710400004A
S11305301148004711480047114800471148004737
S11305401148004711480047114800471148004727
S11305501148004711480047114800471148004717
S11305601148004711480047114800471148004707
S113057011480047114800473105000035050000C7
S1130580390500003D050000410500004505000057
S1130590CD730000E5730000FD73000015740000C6
S11305A01D8000003D8000005590000095900000E3
S11305B0198800003D8800009174000061880000E3
S11305C0002934D00123002210B488422CD3012402
S11305D02407A14204D2814202D209011B01F8E797
S11305E0E400A14204D2814202D249005B00F8E750
S11305F0884201D3401A1A434C08A04202D3001B7C
S11306005C0822438C08A04202D3001B9C082243AE
S1130610CC08A04202D3001BDC082243002803D0EC
S11306201B0901D00909E3E7101C10BC704700281E
S113063001D00020C04307B4024802A14018029030
S113064003BDC046D90000000029F0D003B5FFF770
S1130650B9FF0EBC4243891A1847C046002941D04D
S113066010B4041C4C40A44601230022002900D5E8
S11306704942002800D5404288422CD30124240753
S1130680A14204D2814202D209011B01F8E7E4002D
S1130690A14204D2814202D249005B00F8E78842B9
S11306A001D3401A1A434C08A04202D3001B5C0831
S11306B022438C08A04202D3001B9C082243CC088E
S11306C0A04202D3001BDC082243002803D01B09EC
S11306D001D00909E3E7101C6446002C00D5404210
S11306E010BC7047002806D003DB0020C04340083C
S11306F001E08020000607B4024802A140180290DD
S113070003BDC046190000000029EBD003B5FFF774
S1130710A7FF0EBC4243891A1847C0467047C0461B
S11307208446101C62468C46191C634600E0C04691
S11307301FB500F0B3FF002801D40021C8421FBD3B
S113074010B500F0E3FE4042013010BD10B500F0DA
S1130750A5FF002801DB002010BD012010BDC0460C
S113076010B500F09BFF002801DD002010BD012022
S113077010BDC04610B500F013FF002801DC0020B6
S113078010BD012010BDC04610B500F009FF0028BF
S113079001DA002010BD012010BDC0460000000099
S11307A038B50E4B0C4A041C0D1CFFF7EDFF002856
S11307B004D1201C291C01F0B3FD38BD074B064AA7
S11307C0201C291C01F078FA01F0AAFD80231B06E5
S11307D0C018F2E7C046C046000000000000E04137
S11307E010B5041E33D001F021FE9E231B1A962B54
S11307F009DC083884406402640ADBB26402DB0565
S1130800600A184310BD992B0ADD0522121A211C17
S1130810D1400A1C011C1B318C40611E8C411443C5
S1130820052801DD421F9440144A2240610704D088
S11308300F210C40042C00D0043251010AD59F230F
S1130840181AFF2816D09401640AC3B2D6E700230D
S11308500024D3E7D208FF2B03D05402640ADBB28E
S1130860CCE7002A06D08024E40314436402640A1B
S1130870FF23C3E7FF230024C0E7C046FFFFFFFBBD
S1130880F8B55F46564644464D46F0B40C034D0059
S1130890CE0F610A440F2143C40018038046580058
S11308A0400D8246D80F84464046400A530F034306
S11308B0D0006D0D371C83465246664500D1A4E036
S11308C0AF1A002F00DC09E1002A3BD1184300D005
S11308D0EAE0630700D187E00F232340042B00D113
S11308E082E0221DA242A4416442802309191B0410
S11308F00B40371C141C002B00D17CE0CE4B01357F
S11309009D4200D105E1CD4BE40819404807490256
S113091004430B0B002000211B031A0B0B0D6D0568
S11309201B0513436A08C64DFF071D4015436D00A0
S11309306D08291C3943201C3CBC90469946A246AC
S1130940AB46F8BDBC488542C3D0802000040343B5
S1130950382F00DDF0E01F2F00DD24E12020C01B34
S11309601A1C814682405846F84002439446584631
S11309704A469040421E9041FB40624602431F1C7F
S1130980A21A9442A4416442C91B091B141C0B0201
S11309909FD549024F0A002F00D1C8E0381C01F04E
S11309A045FD021C083A1F2A00DDB5E02821091A7A
S11309B0201C9740C84007439440954200DDB2E0B4
S11309C0551B691C1F2900DDDCE01F22551B3B1C45
S11309D0221CAB40CA40AC40651EAC411343CF401F
S11309E01C43391C002574E780231B040B40371C6F
S11309F0002B00D082E7904B4807E4080443C90861
S1130A009D4248D009030B0B84E7AA1A9446002A96
S1130A1000DC98E05046002852D08748854200D137
S1130A2057E78020000403436246382A00DDFCE0D7
S1130A301F2A00DD4AE120226046101A1A1C824057
S1130A408246914658466246D0404A460243904602
S1130A50584652469040421E9041424602436046E8
S1130A60C3401219A242A441644259180919141C22
S1130A70080200D42DE7704B01359D4200D122E1DC
S1130A806E4B60081940012323401C1C0443CB0710
S1130A901C4349081DE7231C0B433AD080231B0346
S1130AA00B431B031B0B35E7013F002F65D1584651
S1130AB0221A9442A4416442C91A091B141C66E711
S1130AC05846184300D104E7012252429444604638
S1130AD0002800D0C5E058460219C3E7002F73D19F
S1130AE0681C4005400D012800DCDEE05A46A21ACD
S1130AF09442BF41C81A7F42C71B380200D489E020
S1130B005A46141BA3459241591A52428F1A6646FB
S1130B1041E700230024FDE6271C283887400024F1
S1130B20954200DC4CE74549AD1A3940D1E6201C1A
S1130B3001F07CFC203034E75A461A43531E9A4194
S1130B40D2B200271CE7002A00D0DCE0681C420572
S1130B50520D012A00DC8DE0374DA84200D1F3E0AC
S1130B605D462A19A242A441644259180919CC07C6
S1130B70520814434908051CABE62F48854200D0AF
S1130B80E6E6A6E62B1C1F3B3A1CDA40131C202980
S1130B906CD03F22551BAF403C43601E84411C4334
S1130BA00021002595E6381C20381A1CC240101C70
S1130BB0202F5DD04022D71BBB405A461A43531EF8
S1130BC09A4102430027DBE6002D3BD01A4DAA458B
S1130BD000D193E080252D047F422943382F00DD86
S1130BE0ACE01F2F00DD29E12025ED1B081C261C8D
S1130BF0A840FE40AC400643651EAC413443F94076
S1130C005D462C1BA34592415B1A5242991A5546E4
S1130C106646BCE6131C3B43141C002B00D0BAE60A
S1130C200027002100250024E5E65A461A43531EF6
S1130C309A41D2B2002314E7FF070000FFFF7FFFB1
S1130C40FFFF0F800D1C254358D0FF43002F51D1C7
S1130C50041BA3459241591A5242891A55466646C5
S1130C6095E69648854200D0DEE632E6002793E713
S1130C700023A2E7081C2043002D00D0C4E0002874
S1130C8000D1F7E05846184300D122E6584602192D
S1130C90A242A441644259180919141C0A0200D43E
S1130CA017E6874B0125194013E6081C2043002D45
S1130CB039D1002871D15946194303D0191C5C4617
S1130CC0664606E600270021002494E660462038A4
S1130CD01A1CC24060469146202800D1ACE0402254
S1130CE0121A93405A461A43531E9A414B461A43CA
S1130CF00023B6E6714DAA4500D06FE7191C5C4687
S1130D0055466646E5E5002D22D10D1C254377D0D6
S1130D10D543002D71D15C445C459241591852422F
S1130D2089185546A4E600284DD15946194300D1E7
S1130D3094E0191C5C466646604DCAE50C43611E8E
S1130D408C41E4B200215BE7051C0021002452E63B
S1130D505A4DAA4554D05542802210040143382DDF
S1130D6000DD81E01F2D00DD92E02022501B0A1CD3
S1130D7084468240201CE8400243904662469440E8
S1130D80601E844142461443E9405C445C45924100
S1130D90CB185242991855466AE65846184300D172
S1130DA097E55846271ABC429241C81A5242801A03
S1130DB0020266D55846041BA3459241591A524271
S1130DC0891A664685E55846184333D04807E4082F
S1130DD004438020C9080003014208D0DD0805420D
S1130DE005D15946CA085C071443291C6646630F9B
S1130DF0C9001943E400314D6BE5304A9245AED148
S1130E00191C5C46554664E5002836D058461843FC
S1130E1010D080254807E408C9082D03044329425B
S1130E20E5D0D8082842E2D15D46EA085C071443BD
S1130E30011CDCE7214D4CE5002353E73D1C203D1C
S1130E400A1CEA40151C202F34D04026F71BB94059
S1130E500C43611E8C412C430021D1E680210027E4
S1130E60C903164D0024C6E50C43611E8C41E4B24F
S1130E7000218AE7191C5C462BE5191C5C460F4DC2
S1130E8027E5031C3B4300D11CE7011C3C1C20E567
S1130E902020404240190A1CC2409046202D0BD00D
S1130EA04020451BA9400C43611E8C4145462C4300
S1130EB000216AE70021CBE70021F4E7FF070000E7
S1130EC0FFFF7FFFF0B5564644465F464D46F0B4FB
S1130ED01F1C0B031B0B98464B0087B0041C814658
S1130EE05B0DC80F161C9A460090002B51D06A4B1C
S1130EF09A4531D08022414652030A43630FD200FF
S1130F001A43664B90460025E20091469A44002419
S1130F1002953B031B0B9B46FD0F7B00311C5B0DB5
S1130F20019560D05C4A934254D0802158464903CD
S1130F300143720FC9001143584A8B469B18F100B4
S1130F400020009A04436A4003920F2C00D9ADE0BC
S1130F50534EA4003459A746404604436ED10021A1
S1130F6002250824884689460295D2E7009C029807
S1130F70C34649460194022864D0032800D1ABE259
S1130F80012800D038E2019A002402400025A1463D
S1130F9060E0434623434AD04046002800D1C0E1E4
S1130FA001F044FA031E272B00DDB3E128210D1ABA
S1130FB0211C083B4246E9409A400D1C1543221C63
S1130FC09A40A8469146374B00251B1A9A4600249E
S1130FD002959EE75A4616430320002EB1D1B3462C
S1130FE000210220ADE75A4632431BD05B46002B5A
S1130FF000D18AE1584601F019FA272800DD7DE185
S11310002822171A011C321C08395B46FA408B400F
S1131010171C1F43331C8B40BB46191C214B1B1A46
S113102000208EE70027BB460021012089E700202D
S1131030012504248046814602956AE703250C2491
S1131040029566E7019C0394039D01222A40002433
S1131050114DA146002000212403260B0C0D24056C
S1131060114B34432D0523402B435B005B08D2070F
S1131070191C4846114307B03CBC90469946A24609
S1131080AB46F0BD0022802424039146024DE1E7E3
S113109000240025A146DDE7FF07000001FCFFFF57
S11310A058B900000DFCFFFFFFFF0F805546ED1AF5
S11310B00495D84500D953E100D14EE1049C0025A4
S11310C0013C4E4604944746A946584603020C0E7A
S11310D01C430902250C23041B0C0091381C291CF9
S11310E00193FFF76DFA019983464143381C8A4600
S11310F0291CFFF7A9FA330C090419438A450CD9B2
S11311005B460919013B8C4200D947E18A4500D866
S113111044E102225242934409195346CB1A181C43
S1131120291C9846FFF74CFA071C0198291C7843A0
S113113082464046FFF788FA36040B04360C3343E4
S11311409A4509D91B197A1E9C4200D924E19A4573
S113115000D821E1023F1B195E4632041743380CC4
S1131160BB46009E009F51463F0C32045B1A594611
S1131170BA46120C0F043F0C904651467A434F4333
S11311804146414356467043CF19160CBE19B1422D
S113119002D980277F02C019310C12043604120CC4
S11311A04018B618834200D2C4E000D1BEE0191A38
S11311B04846861BB145BF417F42CF1BA74200D1A1
S11311C013E1291C381CFFF7FBF9019902904143F4
S11311D0381C8946291CFFF737FA330C09041943D4
S11311E089450CD9029B0919013B8C4200D9FFE0C7
S11311F0894500D8FCE0029F0919023F02974F4637
S1131200CF1B381C291C0597FFF7DAF9071C019836
S1131210291C784381460598FFF716FA3604090419
S1131220360C0E43B14509D936197B1EB44200D998
S1131230E0E0B14500D8DDE0023F3619029D4946A1
S1131240761A290439430B0457460A0C1B0C4046F2
S11312504546584355437B437A43EB18070CDB1947
S11312609D4202D980256D0252191D0C00041B04F5
S1131270000C52191B18964235D300D1FCE001230F
S11312801943049E994FF519002D00DCA1E048078D
S113129009D00F230B40042B05D00B1D8B42894131
S11312A049428B44191C5A46D20107D5904B5C46DF
S11312B0049E80271C40FF00A346F5198D4B9D42D8
S11312C07ADD039C0122224000248B4DA146C1E615
S11312D080242403474627424CD13C432403240B57
S11312E0009A854DB6E63619481EB4425ED9011CF3
S11312F09642C4D1009E9E42C1D1C2E7031C283B42
S1131300311C99408B46002188E6301C01F08EF890
S1131310203072E6283B211C9940002288469146E1
S113132051E6201C01F082F820303BE60021B14553
S113133000D33DE7009F5A46B944B945BF417F42B7
S11313403F19FB18013A9C421ED2984200D97EE014
S113135000D1B5E0191A93462AE7894500D8ADE6CD
S11313604846464642467708D3074608C0071E4308
S11313708146AAE65846204212D1044324032A1C7B
S1131380240B89465C4D65E6A342E3D1009F4F459B
S1131390DBD9211A93460BE7171CDDE69B46BCE616
S11313A03C432403240B009A534D53E6B24259D8CC
S11313B000D18AE0011C62E75F46C9087B07039EEF
S11313C00B437C026D0501229946240B6D0D3240BE
S11313D040E64A4B049FDB1B382B10DD039C0122A3
S11313E0224000240025A14634E60121494248E771
S11313F0029304E71F1C21E7019C039441E71F2B80
S113140040DC3F48049F0C1C3A1858469140DC408D
S1131410904020430A1C511E8A41011C11435A4624
S1131420DA40131C480709D00F220A40042A05D0C9
S11314300A1D8A42894149425B18111C1A0234D59B
S1131440039C0122224000240125A14602E6009FBC
S113145002214942B9448B44B94589414942091999
S1131460CB18A4E6009D881E6900A942AD416D42D7
S11314702C19361900913AE7002B00D033E70024E9
S1131480009437E71F4A049C5D46121BD5402A1C72
S1131490202B1FD01C4E5F46A3199F403B1C1943B1
S11314A04B1E994111430023BCE75A07C9080A435C
S11314B0039F91465B0201221C0B3A400025C9E5BB
S11314C04E45C4D89346002172E6009F9F42C9D37B
S11314D0011C0FE70023E2E7802424035F463C431A
S11314E02403240B019A8946034DB3E5FF0300004E
S11314F0FFFFFFFEFE070000FF07000002FCFFFFE6
S11315001E040000E2FBFFFF3E040000F0B55F464E
S113151056464D464446F0B40D1C041C8046E80F64
S1131520814618030F03000B3F0B83B084461B480E
S1131530009749005E00DF0F490D9246760DBB46C9
S113154081420CD01548864210D00120B14215D0FA
S113155003B03CBC90469946A246AB46F0BD009F02
S113156001202743F4D10D488642EED16046024360
S11315700120002AECD10120B142E9D1009B63454E
S1131580E6D1D045E4D1D94506D00029E0D11C43A9
S1131590201C441EA041DBE70020D9E7FF07000020
S11315A0F0B55F4656464D464446F0B4CD0FDE0FC7
S11315B0AC461D032D0BB146374E0F034C00AB4612
S11315C05D0080463F0B640D92466D0DB44232D0EF
S11315D0314EB54235D0002C0ED138434142414101
S11315E0081C002D0BD0002919D1CC452DD06546FF
S11315F068420123184318E0002DF6D1281C5946EF
S11316000A4353425341002806D1002BEDD06346D0
S113161058420123184308E00020002B05D14A4614
S1131620504250414042012318433CBC90469946E5
S1131630A246AB46F0BD3E1C0643C9D00220404240
S1131640F3E75E461643C6D0F8E7AC4207DC0BDA94
S1131650614648424841404201231843E5E7664653
S1131660704201231843E0E75F450AD80ED00020FA
S11316705F45DAD265466842684140420123184317
S1131680D3E76246504201231843CEE7D045F8D849
S11316900020D045EED3C8E7FF070000F0B556465A
S11316A04D4644465F46F0B40D1C83B0041C0190C3
S11316B0E80F814618030F03000B3F0B844635489F
S11316C0009749005E00DF0F490D9246760DB8463B
S11316D0814234D02F48864236D0002918D0002EBB
S11316E01FD1341C67463A4353425341002C1FD048
S11316F00020002B05D14246504250414042012374
S1131700184303B03CBC90469946A246AB46F0BD94
S11317100098044360426041041C002EE2D000287B
S1131720E9D1C14515D04F46784201231843E8E773
S1131730002BF6D04B46584201231843E1E7009FA3
S113174002202743DDD1C5E7674602201743D8D1DD
S1131750C3E7B14204DD4A46504201231843D0E7AF
S1131760B14207DB00986045E4D80AD0009F00200E
S11317706745C6D24F467842784140420123184318
S1131780BFE7019A5245D5D8019A00205245F1D3BA
S1131790B7E7C046FF070000F0B5564644465F462B
S11317A04D46F0B41F1C0B031B0B9A464B0087B02D
S11317B0041C80465B0DC80F161C02938146002B47
S11317C068D0694B0299994232D080225346520321
S11317D01A43D200630F1A439246644AE000891800
S11317E080460291002400253B031B0B9B46780096
S11317F0FB0F321C400D039300D175E05A4B984205
S113180069D08022594652030A43730FD2001A4307
S1131810564B9346C018F200002303994E4671407C
S11318201C430F2C00D9A9E0514EA4003459A746FB
S113183053461C4300D087E00025AA46A846082446
S11318400225D1E74946022D6CD0032D00D117E2C1
S1131850012D00D058E10D40EDB20024A94600232B
S1131860A0460020002125030A0D1C052D0B12059E
S1131870404B2A43134023435B004C465B08E2077A
S1131880191C4046114307B03CBC90469946A246F9
S1131890AB46F0BD5346234350D05346002B00D1F2
S11318A084E1504600F0C2FD031E272B00DD76E1E3
S11318B028210D1A211C083B5246E9409A400D1C70
S11318C01543221C9A40AA4690462B4B00241B1A0F
S11318D00293002588E75B461E430323002E9CD118
S11318E0B3460022022398E75B46334321D058468F
S11318F0002800D14EE100F099FD272800DD42E1E7
S113190028210F1A021C311C083A5B46F940934007
S11319100F1C1F43331C9340BB461A1C164B181A4A
S113192000237AE701230B4000249946A0460E4B7E
S113193097E70027BB46002201236EE70021042419
S11319408A46884601254FE70C2403254CE70025E9
S11319508024A9462403A846034B82E7DA4690462E
S113196003991D1C6FE7C046FF07000001FCFFFF41
S113197098B90000FFFF0F800DFCFFFF029F160CBB
S1131980381804904046070C0004000C1204120C92
S1131990031C5343041C3D1C7443554398463B1C91
S11319A073436419A44644460293230C63449D4242
S11319B004D9029D802464022D1902951D0C0395FF
S11319C045462C041B04240C1C1905945C46230C6A
S11319D0051C58432404240C8446381C6043654386
S11319E05F438146CC44280C6044BB46814502D900
S11319F080277F02BB442D04070C2D0C00044019E2
S1131A005546BC462F04E3448446280C3D0C2F1C49
S1131A105743B8462F1C77434243B94647463F0CC9
S1131A209144BA46D14446434A4502D980225202DF
S1131A30B6184F463A0CB6183A0447463F043F0CD2
S1131A40B8462F1C67435D434443584365190190CE
S1131A50380C2D184244B846AC4204D9019880236E
S1131A605B02C0180190039C029F201C6044C019B3
S1131A706045A44147466442A4462B043C0499466D
S1131A80240C4C44A046D8448018C246E2449042F8
S1131A909241574652429146F219E245BF417F4274
S1131AA04B46BC46D845BF41D4187F4263461F43CA
S1131AB02D0C7F19B24292414C45AD4152426D42C8
S1131AC01543019E7D19AB19E20D5B02059F13437B
S1131AD042023A439A46531E9A41C30D101C1843BE
S1131AE06402204380465046C0010DD5454601227C
S1131AF05646049C6B082A401A43F30701341A43E0
S1131B00760804949046B246049E634FF319002B62
S1131B1061DD404640070BD00F2244462240042A90
S1131B2006D04246043242458041404282449046B7
S1131B305546ED0107D5594B5646049F80201E405B
S1131B40C000B2463B18564A934200DDEAE64446DA
S1131B505546E2086807104301226C025B050A40FF
S1131B608046240B5B0D91467BE6DA4690461D1CAD
S1131B7069E680242403574627421CD13C432403AE
S1131B80240B484B6DE6031C283B311C99408B46C3
S1131B900022C3E6301C00F049FC2030ADE6283BAF
S1131BA0211C994000228A4690468EE6201C00F0B3
S1131BB03DFC203078E65846204207D1044303997F
S1131BC02403240B89469046364B4AE63C432403BF
S1131BD0240B344B45E6344B049E9B1B382B06DD0B
S1131BE001230B4000249946A046002339E61F2B0D
S1131BF025DC049C2D4D46466019524644468640D9
S1131C00DC4082405746301C2243DF40441EA04142
S1131C1002433B1C540709D00F201040042805D070
S1131C20101D9042924152429B18021C1D021AD56B
S1131C3001230B4000249946A046012311E61C48C9
S1131C40049C5546001BC540281C202B16D0194E59
S1131C505746A21997403A1C43461A43531E9A41C9
S1131C6002430023D6E758075B02D2081C0B01236A
S1131C700B401043994680460023F2E50022EBE72F
S1131C808024240350460123044319402403240BD5
S1131C908946044BE5E5C046FF030000FFFFFFFE55
S1131CA0FE070000FF07000002FCFFFF1E04000007
S1131CB0E2FBFFFF3E040000F8B55F46564644468B
S1131CC04D46F0B40C034D00CF0F610A440F21437D
S1131CD0C4001803DE0F8046B44646465800760A10
S1131CE0530F3343D600D14A6D0DBA46400DB34667
S1131CF0904200D1F5E06246012672409446674561
S1131D0000D1ABE02F1A002F00DC11E100283ED1F6
S1131D105846184300D0F1E0600700D197E00F2344
S1131D202340042B00D122E1221DA242A44164429B
S1131D30802309191B04012750460B400740141C3B
S1131D40002B00D179E0B94B01359D4200D10BE164
S1131D50B74BE40819404807490204430B0B002021
S1131D6000211B031A0B0B0D6D051B0513436A0899
S1131D70B04DFF071D4015436D006D08291C394304
S1131D80201C3CBC90469946A246AB46F8BDA748E9
S1131D908542C1D0802000040343382F00DDFDE0DC
S1131DA01F2F00DD31E12020C01B1A1C5E4682403B
S1131DB0FE40324394465A468240101C421E9041D3
S1131DC0FB40624602431F1CA21A9442A44164428F
S1131DD0C91B091B141C0A029ED549024F0A002F75
S1131DE000D1D6E0381C00F021FB021C083A1F2A5F
S1131DF000DDC3E02821231C091A9740CB401F4370
S1131E009440954200DDC0E0551B691C1F2900DD8C
S1131E10EAE01F22551B3B1C221CAB40CA40AC40CD
S1131E20651EAC411343CF401C43391C002573E7A6
S1131E3080217E4D0027C90300247C4B4807E40819
S1131E400443C9089D4250D009030B0B87E7802344
S1131E501B04012752460B40174071E72A1A944687
S1131E60002A00DCA1E0002854D07048854200D14B
S1131E7052E78020000403436046382800DD0EE169
S1131E801F2800DD57E162462020801A1E1C864070
S1131E90B1465E46D6404A4632435E468640904648
S1131EA0301C421E9041424602436046C340121910
S1131EB0A242A441644259180919141C080200D40E
S1131EC02AE75A4B01359D4200D131E1584B600855
S1131ED01940012323401C1C0443CB071C4349081D
S1131EE01AE71E4300D00AE705E7231C0B433BD047
S1131EF080231B030B431B031B0B30E7013F002F05
S1131F006DD15E46A21B9442A4416442C91A091BC6
S1131F10141C60E75846184300D1FDE601267642BA
S1131F20B4446046002800D0D0E05E463219BFE7D2
S1131F30002F00D080E0681C4005400D012800DC23
S1131F40E8E05A46A21A9442BF41C81A7F42C71B0E
S1131F503E0200D498E05846041BA3459241591A06
S1131F6052428F1AE2463AE700230024F7E6802320
S1131F701B04012756460B403740E1E6271C28384E
S1131F8087400024954200DC3EE72949AD1A3940D8
S1131F90C2E6201C00F04AFA203026E75A461A43CB
S1131FA0531E9A41D2B200270EE7002A00D0DEE089
S1131FB0681C4605760D012E00DC90E01B4DA842FE
S1131FC000D1F5E05E463219A242A4416442591898
S1131FD00919CC07520814434908051C9CE6134808
S1131FE0854200D0D9E697E62B1C1F3B3E1CDE4001
S1131FF0331C20296FD03F22551BAF403C43601E49
S113200084411C430021002586E6381C20381E1C10
S1132010C640301C202F60D04022D71BBB405A46FC
S11320201A43531E9A4102430027CDE6FF070000DE
S1132030FFFF7FFFFFFF0F80002D37D0B64DA84272
S113204000D18FE080252D047F422943382F00DD05
S1132050A8E01F2F00DD24E12025ED1B0E1CAE405F
S1132060B046261CFE404246AC401643651EAC41B9
S11320703443F9405A46141BA34592415B1A524219
S1132080991A051CE246A6E6131C3B43141C002BBC
S113209000D0A4E60027002100250024CDE65A46FE
S11320A01A43531E9A41D2B2002300E70D1C254364
S11320B058D0FF43002F51D15A46141BA3459241D7
S11320C0591A5242891A051CE24684E6924885420E
S11320D000D0D1E620E6002790E700239FE7081C04
S11320E02043002D00D0C2E0002800D1EFE0584684
S11320F0184300D110E658460219A242A441644292
S113210059180919141C0A0200D405E6834B012549
S1132110194001E6081C2043002D38D100286FD156
S11321205946194303D0191C5C46E246F4E50027DE
S11321300021002481E6604620381A1CC24066460D
S1132140101C202E00D1AAE04022921B93405A4634
S11321501A43531E9A4102430023A8E66E4DA84237
S113216000D073E7191C5C46051CE246D4E5002D3B
S113217022D10D1C254376D0D543002D70D15C446B
S11321805C459241591852428918051C96E600286C
S11321904CD15946194300D14AE6191C5C46E24623
S11321A05D4DB9E50C43611E8C41E4B2002161E749
S11321B0051C0021002440E6574DA84253D0554247
S11321C0802216043143382D7BDC1F2D00DD8CE08A
S11321D02022561B0A1CB446B240261CEE40324351
S11321E0904662469440661EB44142461443E94018
S11321F05C445C459241CB1852429918051C5DE63B
S11322005846184300D187E55E46A71BBC4292415D
S1132210C81A5242801A060260D55846041BA345C8
S11322209241591A5242891AE24675E558461843B2
S113223033D04807E40804438020C908000301425E
S113224008D0DD08054205D15946CA085C07144385
S1132250291CE246630FC9001943E4002E4D5BE5D7
S11322602D4A9042AFD1191C5C46051C54E5002848
S113227030D05846184310D080254807E408C908D0
S11322802D0304432942E5D0D8082842E2D15D4613
S1132290EA085C071443011CDCE71F4D3CE50023FE
S11322A055E73D1C203D0E1CEE40351C202F2ED042
S11322B04026F71BB9400C43611E8C412C4300217E
S11322C0D8E60C43611E8C41E4B2002190E7191C4E
S11322D05C4621E5191C5C460F4D1DE5031C3B4380
S11322E000D124E7011C3C1C16E520267642761911
S11322F00A1CF2409046202D0BD04026751BA940A5
S11323000C43611E8C4145462C43002170E700219B
S1132310D1E70021F4E7C046FF070000FFFF7FFF7D
S113232070B50B1C124C09030E0B5900021C490D0D
S1132330DD0F0020A14211DD0E4881420FDC802018
S1132340400306430C48401A1F280BDD0B4A521A5F
S1132350D640321C5042002D00D1101C70BD084BD9
S1132360E818FBE7074BC240C9188E403243F1E737
S1132370FE0300001D0400003304000013040000E9
S1132380FFFFFF7FEDFBFFFF43001B0E5A1C4102C2
S1132390D2B270B54C0AC50F012A17DDE0229200B3
S11323A06407090B9818002200231E0D221C340513
S11323B00C431B494005400821400143490049089A
S11323C0ED070B1C2B43101C191C70BD002B15D1E1
S11323D0002C1CD0201C00F029F80A281ADC0B2140
S11323E0091A231CCB40191C031C15339C400D4BAC
S11323F00903181A4005090B400DD4E7002C03D03B
S11324006407090B0848CEE707480021CBE7002002
S11324100021C8E7011C0B398C40211C0024E6E78D
S1132420FFFF0F8089030000FF0700001C21012328
S11324301B04984201D3000C10391B0A984201D3A3
S1132440000A08391B09984201D30009043902A281
S1132450105C40187047C0460403020201010101E8
S1132460000000000000000090B587B002AFF860E3
S1132470B9607A603B6005483968FA68BB687C6873
S1132480009400F033F800BEFDE7C046909F0000C2
S113249080B584B000AFF860B9603B60FB1D1A7072
S11324A0FB1D1B78002B06D109490A4A0A4B081C5C
S11324B06921FFF7D9FFF868FB1D1978BA683B68F2
S11324C000F0E8F9031C181CBD4604B080BDC046EA
S11324D0D09F0000D8B90000F49F000080B500AF81
S11324E000F0FCF90023181CBD4680BD0FB480B574
S11324F0A4B000AF00238C22D219136000238822D9
S1132500D21913603B1D1A1C8023101C00211A1CB5
S113251007F02DFD3B1C9C338422D21913609823B1
S1132520DB1918688422D21911683A1D0E4B00F089
S1132530B3FA031C8C22D21913608C22D2191368AB
S11325403A1D101C191C00F0CFF9031C8822D21963
S113255013608822D2191368181CBD4624B080BCAD
S113256008BC04B01847C0466D25000080B586B08D
S113257000AFF860B9603B60FB1D1A7000237B61FB
S113258000237B611DE0BB681B6801337F2B09D9E5
S1132590BB681B68FA68101C191C00F0A5F9BB681D
S11325A000221A60BB681B68FA68D318FA1D1278F7
S11325B01A70BB681B685A1CBB681A607B690133BC
S11325C07B617A693B689A42DDDBBD4606B080BD1B
S11325D080B582B000AF78600A1CFB1C1A70FB1C2B
S11325E01B78002B08D07B68DB78DBB2082213430E
S11325F0DAB27B68DA7007E07B68DB78DBB208224A
S11326009343DAB27B68DA70BD4602B080BDC0463F
S113261080B582B000AF78600A1CFB1C1A70FB1CEA
S11326201B78002B08D07B68DB78DBB204221343D1
S1132630DAB27B68DA7007E07B68DB78DBB204220D
S11326409343DAB27B68DA70BD4602B080BDC046FF
S113265080B582B000AF78600A1CFB1C1A70FB1CAA
S11326601B78002B07D07B689B68802212031A43D7
S11326707B689A6005E07B689A68034B1A407B6824
S11326809A60BD4602B080BDFFFFF7FF80B582B0FF
S113269000AF78600A1CFB1C1A70FB1C1B78002B13
S11326A007D07B689B688022D2021A437B689A60B9
S11326B005E07B689A68034B1A407B689A60BD46C4
S11326C002B080BDFFFFFBFF80B58AB000AFF860A9
S11326D0B9607A603B60FB68002B06D12C492D4A17
S11326E02D4B081CF021FFF7BFFEFB681A792B4B1A
S11326F01A71FB681A68294B1A60284B1B79022B44
S113270023D0062B01D0012B3FD13B1C2033181CB6
S113271006F07EFE3B1C2033BA681A601F4B196812
S11327203A1C20327B68081C111C1A1C06F038FD68
S11327301A4B1B68181C0121FFF74AFF174B1B6833
S1132740181C0121FFF764FF1FE03B1C1433181C05
S113275005F03AFF3B1C1433BA681A600F4B196832
S11327603A1C14327B68081C111C1A1C05F098FDD5
S11327700A4B1B68181C0121FFF76AFF074B1B68F3
S1132780181C0121FFF782FFC046BD460AB080BD78
S113279020A00000E8B9000038A000008CE0FF1F72
S11327A080B500AF124B1B79002B01D100231BE035
S11327B00F4B1B79022B09D0062B01D0012B0BD117
S11327C00B4B1B68181C06F003FE09E0084B1B6842
S11327D0181C05F0C5FE03E0054B00221A71C04623
S11327E0034B00221A710023181CBD4680BDC0464D
S11327F08CE0FF1F80B586B000AFF860B960FB1DA8
S11328001A7000237B61224B1B79022B1DD0062BEF
S113281001D0012B33D1FB1D1B78002B09D01C4B9D
S11328201968FA68BB68081C111C1A1C06F02CFEF7
S113283028E0174B1968FA68BB68081C111C1A1C9D
S113284006F040FE031C7B611CE0FB1D1B78002B83
S113285009D00F4B1968FA68BB68081C111C1A1CB4
S113286005F036FF0EE00A4B1968FA68BB68081CCD
S1132870111C1A1C05F05AFF031C7B6102E00123A2
S11328807B61C0467B69181CBD4606B080BDC0464E
S11328908CE0FF1F80B586B000AFF8607A603B60C3
S11328A03B1C0B330A1C1A70FA683B1C10331A6069
S11328B03B1C10333A1C0B3212781A71391C10313C
S11328C07A683B68081C111C1A1C0023FFF7FCFEE5
S11328D00023181CBD4606B080BDC04680B500AFBD
S11328E0FFF75EFFBD4680BD80B582B000AF786063
S11328F039607B68002B07D109484023191CFF313C
S1132900084A094BFFF7B0FD7A683B68101C191C94
S113291000F00CF8031C181CBD4602B080BDC04674
S113292044A00000F0B900005CA0000080B584B0B1
S113293000AF786039603B1C0F3300221A703B688B
S1132940002B17D07B68002B14D03B1C0F330122C3
S11329501A703B1C0F331B78002B0BD07A683B6832
S1132960101C191C0122FFF745FF031C002B01D08A
S113297000233B603B68181CBD4604B080BDC046C4
S113298080B58CB000AFF860B9607A603B6000231A
S1132990FB61FB68BB61BB695A1CBA6100221A70F7
S11329A07B68002B36D0BB681B68FB62FB6A002B7C
S11329B007D1BB6930221A70FB690133FB61FB69E3
S11329C066E023E0F86A3968FDF748FE031C7B6182
S11329D07B693A685343FA6AD31ABB62BB6A002B19
S11329E006DABB6A3B623B6A3022D31ABB6202E05E
S11329F0BB6A3033BB627B69FB62BB695A1CBA6138
S1132A00BA6AD2B21A70FB690133FB61FB6A002B0C
S1132A10D8D13CE0BB681B687B627B6A002B07D182
S1132A20BB6930221A70FB690133FB61FB692FE03B
S1132A302AE03B68786A191CFDF7C2FD031C3B6160
S1132A403B683A6953437A6AD31A3B623B6A092B5F
S1132A5003D83B6A30333B620BE03B1C38331B78B2
S1132A60002B01D0412300E061233A6A9B180A3B02
S1132A703B623B697B62BB695A1CBA613A6AD2B257
S1132A801A70FB690133FB617B6A002BD1D1FB69AE
S1132A90181CBD460CB080BD90B59DB002AFF86067
S1132AA0B9607A603B6000233B660023FB6500232A
S1132AB0BB613B1C4A3300221A7000233B61FB6854
S1132AC07B6698E17B6C252B0CD07B6CDBB2796840
S1132AD03A1C18325BB23C68081C111C1A1C0123F6
S1132AE0A04785E13B1C4B3301221A7000237B6510
S1132AF00023BB651CE07B6E01337B667B6E1B7819
S1132B005BB27B647B6C2F2B0DDD7B6C392B0ADC79
S1132B107A6D131C9B009B185B001A1C7B6CD318EA
S1132B20303B7B6504E07B6E013B7B660123BB6528
S1132B30BB6D002BDFD006233B657B6E01337B66C8
S1132B407B6E1B785BB22E2B25D100233B650023C3
S1132B50BB651CE07B6E01337B667B6E1B785BB2CE
S1132B607B647B6C2F2B0DDD7B6C392B0ADC3A6D7F
S1132B70131C9B009B185B001A1C7B6CD318303B06
S1132B803B6504E07B6E013B7B660123BB65BB6D4B
S1132B90002BDFD002E07B6E013B7B667B6E013352
S1132BA07B667B6E1B785BB27B647B6C642B1BD077
S1132BB07B6C692B18D07B6C662B15D07B6C462BF9
S1132BC012D07B6C782B0FD07B6C582B0CD07B6C89
S1132BD06F2B09D07B6C622B06D07B6C702B03D0DF
S1132BE07B6C752B00D0B0E07B6C642B02D07B6CCB
S1132BF0692B19D1BB681A1DBA601B687B613A1C2A
S1132C001C323B1C1433391C4B3109780091101CC5
S1132C10191C01220A23FFF7B3FE031CFB653A1CAF
S1132C201C32FB6DD3183B667B6C582B02D07B6C3B
S1132C30782B20D17B6C782B03D13B1C4B330022A7
S1132C401A70BB681A1DBA601B683B613A1C1C32BF
S1132C503B1C1033391C4B3109780091101C191C92
S1132C6000221023FFF78CFE031CFB653A1C1C3268
S1132C70FB6DD3183B667B6C6F2B08D07B6C622B8F
S1132C8005D07B6C702B02D07B6C752B3BD1BB6861
S1132C901A1DBA601B683B617B6C6F2B08D002DC89
S1132CA0622B0AD018E0702B0CD0752B0FD013E0D8
S1132CB03B1C4A3308221A700EE03B1C4A330222A2
S1132CC01A7009E03B1C4A3310221A7004E03B1CC2
S1132CD04A330A221A70C0463B1C4A331B78391CFB
S1132CE01C313A1C1032381C4B3000780090081C00
S1132CF0111C0022FFF744FE031CFB653A1C1C3226
S1132D00FB6DD3183B66FB6D7A6DD31A79683A1C58
S1132D1018323C68081C111C2022A0473B6E002B73
S1132D2012D00DE03B6E5A1E3A661B7879683A1C45
S1132D3018325BB23C68081C111C1A1C0123A04702
S1132D403B6E1B78002BEDD152E07B6C632B13D1CF
S1132D50BB681A1DBA601B68DBB25BB23B643B6C98
S1132D60DBB279683A1C18325BB23C68081C111C4F
S1132D701A1C0123A0473BE07B6C732B2CD1BB684E
S1132D801A1DBA601B68FB64FB6C002B30D0FB6C13
S1132D90181C07F0F4F8031CFB65FB6D7A6DD31A5D
S1132DA079683A1C18323C68081C111C2022A04780
S1132DB00DE0FB6C5A1CFA641B7879683A1C1832D3
S1132DC05BB23C68081C111C1A1C0123A047FB6C55
S1132DD01B78002BEDD10BE07B6CDBB279683A1CDD
S1132DE018325BB23C68081C111C1A1C0123A04752
S1132DF07B6E01337B667B6E1B785BB27B647B6C82
S1132E00002B00D05EE6BB69181CBD461BB090BD0C
S1132E1080B582B000AF78600A1CFB1C1A70074BA7
S1132E207A689200D3581A69FB1C1B78DA40012394
S1132E301340181CBD4602B080BDC046FCB900005A
S1132E4080B584B000AFBA607B603B1C0F33021CBA
S1132E501A703B1C0E330A1C1A703B1C0F331B7870
S1132E60002B04D03B1C0F331B78262B06D920489B
S1132E70AB2359001F4A204BFFF7F6FA3B1C0E33D5
S1132E801B78C92B07D91A485823191CFF31194A32
S1132E901A4BFFF7E9FA7B68002B06D11448AC23E0
S1132EA05900144A164BFFF7DFFA3B1C0E331B780C
S1132EB00233DAB27B681A707B6801333A1C0F3232
S1132EC012781A703B1C0E331B78002B0DD0BB6894
S1132ED0002B0AD07B68991C3B1C0E331B78BA6804
S1132EE0081C111C1A1C07F039F8BD4604B080BD3B
S1132EF074A0000010BA000088A00000ACA000007C
S1132F00C0A0000080B584B000AF786039600123B0
S1132F10FB600023BB607B68002B06D14148B623CD
S1132F205900414A414BFFF79FFA3B68002B07D1F8
S1132F303C486E23191CFF313B4A3D4BFFF794FA82
S1132F403B689B68002B06D13648B7235900364AA4
S1132F50384BFFF789FA7B681B7D1A1C7B689B69D9
S1132F60DBB2101C191CFFF753FF031C002B07D105
S1132F702C487223191CFF312B4A2F4BFFF774FA8C
S1132F807B681433BB607B681A1C0C322B4B101CFF
S1132F9001211A1C00F046F9031CFB60FB68002B9E
S1132FA015D1BB681B781A1CBB685B68DBB2101CAC
S1132FB0191C012201F0AEFF7B681A1C0C321F4B56
S1132FC0101C00211A1C00F02DF9031CFB60FB6887
S1132FD0002B08D17B681A683B68101C191C02F08E
S1132FE011F8031CFB60FB68002B0AD17B681A1CD8
S1132FF00C32124B101C01211A1C00F013F9031C93
S1133000FB60BB681B781A1CBB685B68DBB2101CD6
S1133010191C012201F0BAFFFB68181CBD4604B05C
S113302080BDC04674A0000020BA0000D8A00000F3
S1133030F0A000000CA1000028A10000404B4C00AF
S113304080B588B000AFF860B9607A600123FB6195
S1133050FB681433BB613B1C173300221A70FB68F6
S1133060002B07D16748A223191CFF31664A674B1E
S1133070FFF7FAF9BB68002B06D16248D123590047
S1133080614A634BFFF7F0F9BB689B68002B07D1DB
S11330905C48A423191CFF315B4A5E4BFFF7E4F93B
S11330A0BB691B781A1CBB695B68DBB2101C191C5A
S11330B0FFF7AEFE031C002B07D15248A623191CB0
S11330C0FF31514A544BFFF7CFF9BB689A683B1C58
S11330D017331A70BB681A68BB689B68101CFF2101
S11330E01A1C06F044FFFB681A1C0C327B68101C87
S11330F000211A1C00F096F8031CFB61FB69002BED
S113310016D1BB691B781A1CBB695B68DBB2101C47
S1133110191C012201F0FEFEBB6801229A60FB68C3
S11331201A68BB68101C191C01F06CFF031CFB61BE
S1133130FB69002B1DD1BB685B681B781A1CBB683C
S11331409A60BB689A683B1C17331B789A4203D871
S1133150BB689B68002B0CD1BB691B781A1CBB692C
S11331605B68DBB2101C191C012201F00FFF2B4B12
S1133170FB61FB69002B26D1BB689B685A1EBB68A8
S11331809A60BB681B685A1CBB681A60BB685B68A2
S11331905A1CBB685A60FB681A68BB68101C191C6F
S11331A001F030FF031CFB61BB689B685A1CBB68C1
S11331B09A60BB681B685A1EBB681A60BB685B6870
S11331C05A1EBB685A60FB69002B0AD1FB681A1CA3
S11331D00C32134B101C01211A1C00F023F8031CA1
S11331E0FB61BB691B781A1CBB695B68DBB2101CF2
S11331F0191C012201F0CAFEFB69181CBD4608B067
S113320080BDC04674A0000030BA0000D8A0000001
S1133210F0A000000CA1000094A10000252C0000E7
S1133220404B4C0080B586B000AFF8607A603B1C20
S11332300B330A1C1A703B1C133300221A70002330
S11332407B61FB68002B06D12248F6235900224AF1
S1133250224BFFF709F97B68002B03D07A68204BD7
S11332609A4206D91B48F72359001B4A1D4BFFF706
S1133270FBF8FB681B781A1CFB685B68DBB2101C4C
S1133280191CFFF7C5FD031C5A1E9341DAB23B1CFF
S113329013331A707B6964337B61642001F040FD51
S11332A03B1C13331B78DBB21A1C3B1C0B331B78FF
S11332B09A4203D07A687B699A42DAD87A687B6941
S11332C09A4201D9002300E0074B181CBD4606B002
S11332D080BDC04674A0000044BA0000D8A100001C
S11332E0FFE0F505F0A10000262C000080B58AB0AF
S11332F000AFF8607B603B1C0B3319703B1C0A3336
S11333001A7000237B623B1C14337A681A603B1CDE
S113331014333A6B5A603B1C0B331A783B1C14333E
S11333209A603B1C14330022DA60FB68002B06D140
S11333302C48832399002C4A2C4BFFF795F83B1C0F
S11333400B331B78002B05D126482949264A294BE3
S1133350FFF78AF87B68002B05D122482649224AC8
S1133360264BFFF781F8FA683B1C1433101C191C18
S1133370FFF7C8FD031C7B627B6A002B01D07B6ACC
S11333802CE03B1C0A331B78002B26D03B6B002B14
S113339005D114481A49144A1A4BFFF765F83B1C27
S11333A00A331A783B1C14339A60F9683A1C1432B5
S11333B07B6B081C111C1A1CFFF742FE031C7B626A
S11333C07B6A002B09D13B1C14335B68FA68101C20
S11333D0191C00F019F8031C7B627B6A181CBD469B
S11333E00AB080BD74A0000054BA0000D8A0000048
S11333F00D0200001CA200000E0200002CA200001E
S11334001D02000048A2000080B582B000AF7860C1
S113341039607B68002B05D111481249124A134BBD
S1133420FFF722F83B68002B05D10D4810490E4ADE
S1133430104BFFF719F83B6802331A787B681A7748
S11334403B6801331A787B685A777B685B7F002B73
S113345001D1002300E0084B181CBD4602B080BD1A
S113346074A00000D502000068BA0000D8A00000D3
S1133470D6020000E4A20000242C000080B586B02F
S113348000AFF860B960FB1D1A7001237B61FB6813
S1133490002B05D122482349234A244BFEF7E4FF9D
S11334A0BB68002B05D11E4821491F4A214BFEF75A
S11334B0DBFFBB685B68002B06D11948BA2399006F
S11334C0194A1D4BFEF7D0FFFB681A78BB681A70C7
S11334D0BB681B78033BDAB2BB681A70BB681B7805
S11334E0FA1D12789A4202D2144B7B6101E0002348
S11334F07B617B69002B0ED1BB681B78002B0AD043
S1133500BB685968FB68DA1CBB681B78081C111C73
S11335101A1C06F023FD7B69181CBD4606B080BD4D
S113352074A00000E60200007CBA0000E4A20000DF
S1133530E702000000A300001CA30000252C0000EB
S113354090B589B002AFF8607B603B1C0B331970F7
S11335503B1C0A331A70F8683B1C0B3319783B1C6C
S11335600A331A787B68BC6A0094FC6A0194FFF7FA
S1133570BDFE031C7B617B69002B08D1BB6A1B78F1
S11335803A1C0A3212789A4201D0034B7B617B6960
S1133590181CBD4607B090BD252C0000B0B586B000
S11335A002AF786039600023FB603B1C0B330022C0
S11335B01A707B68002B06D13448DA239900344A08
S11335C0344BFEF751FF3B68002B05D12F4832499D
S11335D02F4A324BFEF748FF7B6801221A777B683B
S11335E000225A777B681A1C0C322D4B101C0121C7
S11335F01A1CFFF717FE031CFB60FB68002B05D1A8
S11336007B68181C00F034FA031CFB60FB68002B79
S11336100CD13B1C0B3301221A707A683B1C0B3310
S1133620101C191C00F0B2FA031CFB60FB68002B91
S113363009D13B1C0B331B7801225340DBB2002B16
S113364001D0184BFB60FB68002B10D13B68197844
S11336503B685A783B689B783868C5783868047941
S113366078680095019400F029FB031CFB603B681B
S11336701B787A68101C191C00F0AAFB031CFB6061
S1133680FB68181CBD4604B0B0BDC04674A0000061
S11336908CBA0000D8A000006903000098A30000C1
S11336A0404B4C00272C000080B582B000AF7860FE
S11336B07B68002B06D10C48E52399000B4A0C4B80
S11336C0FEF7D2FE7B6800221A707B6800225A70D3
S11336D07B6800229A707B680122DA707B68002282
S11336E01A71BD4602B080BD74A0000094BA0000F7
S11336F098A3000090B5EFB002AFF8607A603B6029
S1133700AA4BD8204000C019C3180A1C1A70002301
S1133710D6214900C9190B60AC22FF32BB18002224
S11337201A70A24BD8204000C019C3181B78002B74
S113373007D09E4BD8214900C919CB181B78262BDA
S113374005D99B489B499C4A9C4BFEF78DFE7B68A0
S1133750002B06D19648EA239900974A984BFEF726
S113376083FE7B681B78C92B05D991489549924AF9
S1133770954BFEF779FE8D4BD8225200D219D318FF
S11337801B78022B5FD0894BD8204000C019C31886
S11337901B78042B57D0854BD8214900C919CB1865
S11337A01B78052B4FD0814BD8225200D219D31845
S11337B01B78092B47D07D4BD8204000C019C31873
S11337C01B780B2B3FD0794BD8214900C919CB1852
S11337D01B78142B37D0754BD8225200D219D3182A
S11337E01B781B2B2FD0714BD8204000C019C31855
S11337F01B781C2B27D06D4BD8214900C919CB1835
S11338001B781F2B1FD0694BD8225200D219D31812
S11338101B78222B17D0654BD8204000C019C31841
S11338201B78232B0FD0614BD8214900C919CB1821
S11338301B78072B07D05D4BD8225200D219D3181E
S11338401B781D2B04D17B685B68002B00D073E0D0
S1133850564BD8204000C019C3181B78022B5FD0E8
S1133860524BD8214900C919CB181B78042B57D0C7
S11338704E4BD8225200D219D3181B78052B4FD0A7
S11338804A4BD8204000C019C3181B78092B47D0D5
S1133890464BD8214900C919CB181B780B2B3FD0B4
S11338A0424BD8225200D219D3181B78142B37D08C
S11338B03E4BD8204000C019C3181B781B2B2FD0B7
S11338C03A4BD8214900C919CB181B781C2B27D097
S11338D0364BD8225200D219D3181B781F2B1FD075
S11338E0324BD8204000C019C3181B78222B17D0A4
S11338F02E4BD8214900C919CB181B78232B0FD084
S11339002A4BD8225200D219D3181B78072B07D080
S1133910264BD8204000C019C3181B781D2B01D199
S1133920012300E00023002B06D02148EB2399005B
S1133930214A264BFEF798FD1C4BD8214900C91992
S1133940CB181B78012B43D0184BD8225200D21924
S1133950D3181B78032B3BD0144BD8204000C0193C
S1133960C3181B780B2B33D0104BD8214900C9192D
S1133970CB181B78122B2BD00C4BD8225200D21907
S1133980D3181B781A2B23D0084BD8204000C01919
S1133990C3181B781B2B1BD0044BD8214900C91911
S11339A0CB181B781C2B13D0CB2312E05BFEFFFF3C
S11339B074A00000A7030000A8BA000088A00000BB
S11339C0B4A30000A9030000D0A30000F4A30000E6
S11339D00023AC20FF303A1813707B6819787B6899
S11339E05A68214BD8204000C019C31818783B1CD2
S11339F0E033FFF725FA7B681B780233D9B2F86805
S1133A00AC22FF32BB181A783B1CE0333C1C143444
S1133A100094164C0194FFF769FC031CD620400067
S1133A20C01903603B68002B16D0D6214900C91980
S1133A300B68002B10D1391C14313A68E020400087
S1133A403B181B78081C111C1A1CFFF717FD031CDC
S1133A50D6214900C9190B60D6225200D219136825
S1133A60181CBD466DB090BD5BFEFFFF008793033D
S1133A7080B586B002AF78600123FB603B1C08333D
S1133A80012000210022FFF7DBF97A683B1C083390
S1133A900021009108490191101C02210022FFF726
S1133AA025FC031CFB60642001F014F9FB68181C5E
S1133AB0BD4604B080BDC046404B4C0080B586B0C6
S1133AC002AF78603B1C0C33032000210022FFF777
S1133AD0B7F97A683B1C0C33002100910549019128
S1133AE0101C02210022FFF701FC031C181CBD4618
S1133AF004B080BD404B4C0080B58CB002AF786000
S1133B0039603B68002B05D119481A491A4A1B4BE6
S1133B10FEF7AAFC3B681B78002B03D03B685B686C
S1133B20002B05D112481649134A164BFEF79CFC8C
S1133B303B6819783B685A683B1C18330420FFF72C
S1133B407FF93B681B780233DAB279683B1C18337F
S1133B50381C083000900C480190081C111C0322EA
S1133B60FFF7EEFC031C181CBD460AB080BDC0461E
S1133B7074A00000E6030000B8BA0000B4A300007B
S1133B80E70300008CA70000C0E1E40080B58EB01C
S1133B9002AF786039600023BB623A1C0C323F4BA1
S1133BA0111C1A1C0523081C111C1A1C06F0D6F93A
S1133BB03B1C273305221A703B1C2F3300221A703A
S1133BC03B68002B05D136483649374A374BFEF758
S1133BD04BFC3B1C27331B78002B04D03B1C2733A6
S1133BE01B78052B05D92E4831492F4A314BFEF756
S1133BF03BFC3B6800221A703B1C273319783A1CA3
S1133C000C323B1C1C330220FFF71AF93B1C2733F0
S1133C101B780333DAB279683B1C1C33381C14302C
S1133C20009025480190081C0721FFF789FC031C1C
S1133C30BB62BB6A002B2BD13B6801221A703B1C70
S1133C402F3300221A701BE03B1C2F331B780333E5
S1133C503A1C1432D35CDB43DAB23B1C2F331B789F
S1133C60391C0C31CB5C9A4203D03B6800221A7099
S1133C700EE03B1C2F331A783B1C2F3301321A7091
S1133C803A1C2F323B1C273312781B789A42DBD321
S1133C90BB6A181CBD460CB080BDC04678A80000A5
S1133CA074A000007C040000C8BA000034A800001E
S1133CB07D0400004CA80000404B4C0080B588B047
S1133CC002AF7860081C111C1A1CFB1C1870BB1C6A
S1133CD019707B1C1A703B1C173315221A70FB1CBD
S1133CE01B78032B05D92F482F49304A304BFEF758
S1133CF0BBFB7B1C1B78012B05D92A482D492B4A79
S1133D002D4BFEF7B1FB3B1C20331B78012B05D94F
S1133D1024482A49254A2A4BFEF7A6FB3B1C243398
S1133D201B78012B05D91F482649204A264BFEF74C
S1133D309BFB3B1C1733FA1C127815321A703B1C80
S1133D4017331A783B1C1033101C04210022FFF790
S1133D5077F83B1C1033BA1C12789A703B1C103352
S1133D607A1C1278DA703B1C10333A1C2032127819
S1133D701A713B1C10333A1C243212785A717A6837
S1133D803B1C1033391C0831009110490191101C5F
S1133D9006210322FFF7AAFA031C181CBD4606B02D
S1133DA080BDC04674A00000B9040000D8BA000069
S1133DB080A80000BA040000D8A80000BB040000DA
S1133DC004A90000BC0400003CA90000404B4C00C6
S1133DD080B5EAB002AF78600A1C334BD0214900A9
S1133DE0C919CB181A707B68002B05D12F483049AC
S1133DF0304A314BFEF738FB2B4BD0225200D219FC
S1133E00D3181B78002B1DD0274BD0214900C9198A
S1133E10CB181B78032B15D0234BD0225200D21978
S1133E20D3181B78012B0DD01F4BD0214900C91981
S1133E30CB181B78022B05D01C4820491D4A204B67
S1133E40FEF712FB3B1CD433252001210022FEF790
S1133E50F7FF154BD0225200D219D3181B78002B30
S1133E6007D0114BD0214900C919CB181B78022B5C
S1133E7004D13B1CD43302229A7003E03B1CD4339C
S1133E8005229A707A683B1CD433391C083100919E
S1133E900C490191101C03210322FFF751FB031C61
S1133EA0181CBD4668B080BD63FEFFFF74A000000F
S1133EB069060000F4BA0000D8A000006B060000F8
S1133EC03CAA0000404B4C0080B582B000AF786043
S1133ED00A1CFB1C1A70074B7A689200D358FA1C10
S1133EE012780121081C9040021C5A60BD4602B0A1
S1133EF080BDC0460CBB000090B583B000AF7860B5
S1133F00FB1C1970BB1C1A70BB1C1B78002B12D134
S1133F10134B7A689200D358114A796889008A58F9
S1133F205269F91C09780120041C8C40211CC943E6
S1133F300A405A6110E00A4B7A689200D358084A42
S1133F40796889008A585169FA1C12780120041C86
S1133F509440221C0A435A61BD4603B090BDC0463A
S1133F600CBB000080B58AB000AF786039603B6854
S1133F70002B31D13B1C083308229A807B689A6855
S1133F803B1C08331A603B1C083301229A713B1C0A
S1133F9008330022DA713B1C083300221A723B1CDE
S1133FA0083301225A727B685A683B1C0833DA6072
S1133FB03A1C08323B1C1833101C191C00F056FF25
S1133FC07B6819687B685B683A1C1832081C111CF2
S1133FD01A1C00F0FDFE09E07B6819687B685B68C9
S1133FE03A68081C111C1A1C00F0F2FEBD460AB007
S1133FF080BDC04680B582B000AF78607B68002B7E
S113400006D11549154A164B081C4D21FEF72CFA0A
S11340107B681B781A1C7B685B68DBB2101C191C5C
S11340200022FFF769FF7B681B7A1A1C7B68DB6838
S1134030DBB2101C191C0122FFF75EFF7B681B7AA0
S11340401A1C7B68DB68DBB2101C191CFFF73CFFF1
S1134050BD4602B080BDC046F0AA000020BB0000EF
S113406008AB000080B584B000AF78600A1CBB1CAC
S11340701A803B1C0E3300221A807B685B79012B6B
S113408012D1BB1C1B881BB2002B04DBBB1C1B887E
S11340909B089BB206E0BB1C1B889B089BB2114A81
S11340A013439BB2BA1C13803B1C0E33BA1C1288F8
S11340B01A803B1C0E3300229B5E7A68927953432C
S11340C0181C6421FCF7CAFA031C1A1C3B1C0E338F
S11340D01A803B1C0E331B881BB2181CBD4604B04F
S11340E080BDC04600C0FFFF80B584B000AF7860DB
S11340F039600023FB603B1C0B3300221A703B68C1
S11341001A687B681A603B681A797B681A713B6885
S11341105A797B685A717B6800229A717B68181CF3
S113412000F056FA031CFA681343FB60FA235B00A1
S1134130181C00F0E9FA3B68DB797A68101C191C3A
S113414000F0A4F9031CFA681343FB603B685B7935
S1134150002B01D1022300E000233A1C0B32137020
S11341603B6899793B1C0B333A1C0B3212780A4397
S11341701A703B1C0B333A1C0B32127801210A4390
S11341801A707A683B1C0B331B78101C2A211A1CEA
S113419000F0B0F8031CFA681343FB60FB68181CBA
S11341A0BD4604B080BDC04680B584B000AF786021
S11341B039600023FB603B1C0B3300221A703B1C4C
S11341C00B333A6812781A703B685B78002B01D085
S11341D0102300E000233A1C0B32391C0B31097800
S11341E00B4313707A683B1C0B331B78101C1D2186
S11341F01A1C00F07FF8031CFA681343FB603B6849
S11342005B88181C3F21FCF7DBF9031C9AB23B1CAA
S11342100B331A707A683B1C0B331B78101C1F215C
S11342201A1C7F2300F0E2F8031CFA681343FB60B6
S11342303B681B797A68101C20211A1CFF2300F0AC
S1134240D5F8031CFA681343FB607B68181C0E2125
S11342501022102300F0CAF8031CFA681343FB6011
S1134260FB68181CBD4604B080BDC04680B584B050
S113427000AF786039603B1C0F3300221A700023B2
S1134280BB603B685B78202B06D91749174A184B4B
S1134290081CFA21FEF7E8F83B6819783B685A785D
S11342A03F231340DAB23B1C0F330A431A707A6877
S11342B03B1C0F331B78101C09211A1C00F01AF840
S11342C0031CBB603B689B787A68101C0A211A1C8B
S11342D000F010F8031CBA681343BB60BB68181CD9
S11342E0BD4604B080BDC04614AB000030BB000026
S11342F030AB000080B588B000AF7860FB1C19704B
S1134300BB1C1A703B1C0833181C0021182205F032
S11343102EFE7B681A793B1C08331A713B1C083348
S113432000225A71FB1C1A783B1C08339A603B1C10
S1134330083301221A733B1C0833BA1C1A613B1C54
S1134340083301225A613B1C083300221A607B683F
S11343501A683B1C0833101C191C03F02BFD031CAA
S1134360181CBD4608B080BD80B58AB000AFF860A7
S11343707A601A1C3B1C0B3319703B1C0A331A70ED
S11343803B1C1033181C0021182205F0F0FDFB68BB
S11343901A793B1C10331A713B1C103301225A71D9
S11343A03B1C0B331A783B1C10339A603B1C1033B4
S11343B001221A733B1C10337A681A613B1C0A33BE
S11343C01A783B1C10335A613B1C103300221A60CC
S11343D0FB681A683B1C1033101C191C03F0EAFC20
S11343E0031C181CBD460AB080BDC04680B584B00D
S11343F000AF7860081C111C1A1CFB1C1870BB1C35
S113440019707B1C1A703B1C0B3300221A7000239A
S1134410FB607968FB1C1A783B1C0B33081C111CCD
S11344201A1C0123FFF7A0FF031CFB607B1C1B78F5
S1134430DB43DBB23A1C0B321278D2B21340DBB24C
S1134440DAB23B1C0B331A70BB1C7A1C1B78127833
S11344501340DAB23B1C0B331B781343DAB23B1C18
S11344600B331A703B1C0B331B787968FA1C1278D7
S1134470081C111C1A1CFFF73DFF031CFA681343A8
S1134480FB60FB68181CBD4604B080BD80B582B0DB
S113449000AF78600A1CFB1C1A707B685B79012BE7
S11344A014D1FB1C1B78012B08D0022B0AD0002B43
S11344B000D00BE07B6818229A7107E07B683022F9
S11344C09A7103E07B6861229A71C0467A68FB1C8A
S11344D01B78101C0E211A1CFFF70CFF031C181C60
S11344E0BD4602B080BDC04680B584B000AF7860E0
S11344F0FB1C1970BB1C1A700023FB603B1C0B33A4
S113450000221A703B1C0A33FA1C12781A703B1CE6
S11345100A331B7801229A403B1C09331A703B1C56
S11345200A331B7801229A403B1C0B331A707968BA
S11345303B1C0B331A783B1C09331B78081C2D21B8
S1134540FFF754FF031CFA681343FB60BB1C1A7883
S11345503B1C0A331B789A403B1C0B331A70796856
S11345603B1C0B331A783B1C09331B78081C2E2187
S1134570FFF73CFF031CFA681343FB60FB68181C3D
S1134580BD4604B080BDC04680B584B000AF78603D
S11345900A1CFB1C1A700023FB60FB1C1B78002BFD
S11345A001D0012300E000233A1C0B3213707A6817
S11345B03B1C0B331B78101C2A211A1C0123FFF708
S11345C015FF031CFB60FB68181CBD4604B080BDCE
S11345D080B582B000AF78607B68181C2B21402224
S11345E0FFF788FE031C181CBD4602B080BDC04600
S11345F080B586B000AF7860396000237B613B1CD6
S1134600123300221A807A683B1C0C33101C0121DF
S11346101A1C0623FFF7A8FE031C7B613B1C0C330A
S11346201B781B029AB23B1C0C335B7813439AB27F
S11346303B1C12331A807A683B1C12331B88101CF3
S1134640191CFFF70FFD031C1A1C3B681A803B1C46
S11346500C339B781B029AB23B1C0C33DB7813435C
S11346609AB23B1C12331A807A683B1C12331B88A3
S1134670101C191CFFF7F6FC031C1A1C3B685A801B
S11346803B1C0C331B791B029AB23B1C0C335B7929
S113469013439AB23B1C12331A807A683B1C1233C0
S11346A01B88101C191CFFF7DDFC031C1A1C3B683B
S11346B09A807B69181CBD4606B080BD80B584B065
S11346C000AF021CBB1D1A8002F078FC031C181CEE
S11346D0FA239900FBF774FF031CFB60FB680322B9
S11346E09343FB6009E0FB68181C0438C046FCD106
S11346F0BB1D1A88BB1D013A1A80BB1D1B88002BE9
S1134700F1D1BD4604B080BD80B584B000AF021CB9
S1134710BB1D1A8002F052FC031C181CFA239900DA
S1134720FBF74EFF031CBA1D12885343181CFA23CF
S11347309900FBF745FF031CFB60FB6807229343CA
S113474004221343FB60FB68181C0438C046FCD1E8
S1134750BD4604B080BDC04680B584B000AF78606B
S113476039600023FB603B1C0B3300221A703B684A
S11347701A687B681A603B681A797B681A713B680F
S1134780DA797B685A710220FFF798FF7B68181C5E
S1134790002100F00FF9031CFA681343FB603B6827
S11347A09B79002B01D0802300E000233A1C0B32BC
S11347B013707A683B1C0B331B78101C11211A1CD4
S11347C000F030F8031CFA681343FB603B1C0B3306
S11347D000221A703B1C0B333A1C0B32127818213E
S11347E00A431A703B685B79002B01D0012300E077
S11347F000233A1C0B32391C0B3109780B4313701C
S11348007A683B1C0B331B78101C10211A1C00F017
S113481009F8031CFA681343FB60FB68181CBD46C7
S113482004B080BD80B588B000AF7860FB1C1970FF
S1134830BB1C1A703B1C0833181C0021182205F0FD
S113484096FB7B681A793B1C08331A713B1C0833AE
S113485000225A71FB1C1A783B1C08339A603B1CDB
S1134860083301221A733B1C0833BA1C1A613B1C1F
S1134870083301225A613B1C083300221A607B680A
S11348801A683B1C0833101C191C03F093FA031C10
S1134890181CBD4608B080BD80B58AB000AFF86072
S11348A07A603B603B1C0B330A1C1A703B1C1033B0
S11348B0181C0021182205F05AFBFB681A793B1CCE
S11348C010331A713B1C103301225A713B1C0B33F9
S11348D01A783B1C10339A603B1C103301221A7364
S11348E03B1C10337A681A613B1C10333A685A61D6
S11348F03B1C103300221A60FB681A683B1C1033FF
S1134900101C191C03F056FA031C181CBD460AB0EF
S113491080BDC04680B584B000AF7860081C111C0F
S11349201A1CFB1C1870BB1C19707B1C1A703B1CD6
S11349300B3300221A700023FB607968FB1C1A7881
S11349403B1C0B33081C111C1A1C0123FFF7A4FF8A
S1134950031CFB607B1C1B78DB43DBB23A1C0B3271
S11349601278D2B21340DBB2DAB23B1C0B331A70AA
S1134970BB1C7A1C1B7812781340DAB23B1C0B3335
S11349801B781343DAB23B1C0B331A703B1C0B33FA
S11349901B787968FA1C1278081C111C1A1CFFF782
S11349A041FF031CFA681343FB60FB68181CBD46F7
S11349B004B080BD80B584B000AF78600A1CFB1CD5
S11349C01A70FB1C1B78002B01D0012300E000238C
S11349D03A1C0F3213707A683B1C0F331B78101C7F
S11349E010211A1C0123FFF795FF031C181CBD4658
S11349F004B080BD80B582B000AF78607B68181CBD
S1134A00102102220223FFF785FF031C181CBD4658
S1134A1002B080BD80B584B000AF786039600023F7
S1134A20FB603B1C0B3300221A707A683B1C0B336F
S1134A30101C00211A1C0123FFF72EFF031CFB602E
S1134A403B1C0B331B781A1C082313405A1E93413A
S1134A50DAB23B681A70FB68181CBD4604B080BD0E
S1134A6080B588B000AFF860B9607A603B6000231D
S1134A70FB61FA683B1C1433101C00211A1C06232A
S1134A80FFF70AFF031CFB613B1C14331B781B025A
S1134A909AB23B1C14335B7813439BB29AB2BB6843
S1134AA01A803B1C14339B781B029AB23B1C1433B0
S1134AB0DB7813439BB29AB27B681A803B1C143395
S1134AC01B791B029AB23B1C14335B7913439BB2D0
S1134AD09AB23B681A80FB69181CBD4608B080BDB9
S1134AE080B584B000AF786039600023FB603B1C64
S1134AF00B3300221A707A683B1C0B33101C0F21F5
S1134B001A1C0123FFF7C8FE031CFB603B1C0B337C
S1134B101B78DAB23B681A703B681B78DAB27B68A0
S1134B205B79DBB2D318DBB2DAB23B681A70FB688C
S1134B30181CBD4604B080BD80B582B000AF78605B
S1134B4039603B68012B06D90748FD235900074A01
S1134B50074BFDF789FC7B683A6804329200D3580E
S1134B60181CBD4602B080BD50AB000040BB000025
S1134B7068AB000080B584B000AF021CBB1D1A8076
S1134B80BB1D1B880D4A5343181C0D49FBF718FD28
S1134B90031C1A1C3B1C0E331A803B1C0E331B884F
S1134BA0084A5343181CFA239900FBF709FD031C18
S1134BB09BB2181CBD4604B080BDC046E40C000086
S1134BC0FFFF00007105000090B585B000AF021C26
S1134BD0BB1D1A803B1C0E3300221A803B1C0C3375
S1134BE000221A803B1C0A33BA1D1288D2431A8051
S1134BF03C1C0E343B1C0A331B88181CFFF7BAFFFD
S1134C00031C23803B1C0E331B8864225343181C53
S1134C10C821FBF7D5FC031C1A1C3B1C0C331A805F
S1134C203B1C0C331B88181CBD4605B090BDC04608
S1134C3080B586B000AFF860B9607A6000237B610C
S1134C40F968BA687B68081C111C1A1C02F0AAF8DF
S1134C50FA68BB68101C191C02F0E4F8031C7B61A1
S1134C607A6980231340F3D0FA68BB68101C191CBE
S1134C70FFF762FF031C9BB2181CBD4606B080BD43
S1134C8090B587B000AFF860B9607A603C1C163408
S1134C90F968BA687B68081C111C1A1CFFF7C8FF66
S1134CA0031C23803B1C16331B88181CFFF78CFF46
S1134CB0031C181CBD4607B090BDC04680B582B029
S1134CC000AF02F07BF9031C7B607B68181CBD46B7
S1134CD002B080BD80B584B000AF021CBB1D1A8039
S1134CE0FFF7ECFF031C181CFA239900FBF768FC80
S1134CF0031CFB60FB6803229343FB6009E0FB6831
S1134D00181C0438C046FCD1BB1D1A88BB1D013ACF
S1134D101A80BB1D1B88002BF1D1BD4604B080BD99
S1134D2080B584B000AF021CBB1D1A80FFF7C6FF1C
S1134D30031C181CFA239900FBF742FC031CBA1D40
S1134D4012885343181CFA239900FBF739FC031CFF
S1134D50FB60FB680722934304221343FB60FB6858
S1134D60181C0438C046FCD1BD4604B080BDC04602
S1134D7080B582B000AF78600A1CFB1C1A70074B28
S1134D807A689200D358FA1C12780121081C9040CA
S1134D90021C5A60BD4602B080BDC04660BB000024
S1134DA080B582B000AF78600A1CFB1C1A70074BF8
S1134DB07A689200D358FA1C12780121081C90409A
S1134DC0021C9A60BD4602B080BDC04660BB0000B4
S1134DD080B584B000AFF860B9607A60FB68012BDD
S1134DE006D90F490F4A104B081C3921FDF73CFB2B
S1134DF0BB68002B06D10A490A4A0C4B081C3A210D
S1134E00FDF732FB0A4BFA689200D158BA687B6806
S1134E10081C111C1A1C03F011FFBD4604B080BD10
S1134E2084AB00007CBB0000A4AB0000B4AB00006A
S1134E3074BB000080B582B000AF78607B68002B43
S1134E4006D10749074A084B081C9121FDF70CFBC2
S1134E507B68181C03F0C8FEBD4602B080BDC04686
S1134E6084AB000090BB0000B4AB000080B582B0FE
S1134E7000AF786039607B68002B06D12049214A55
S1134E80214B081CD321FDF7EFFA3B68002B06D118
S1134E901B491C4A1D4B081CD421FDF7E5FA3B684D
S1134EA0181CFFF7C7FF7B689B88082B0AD07B6818
S1134EB09B88102B06D01249124A154B081CDA2184
S1134EC0FDF7D2FA7B681A683B68DA607B689A79E6
S1134ED03B68DA707B68DA793B689A707B681B7A86
S1134EE01A1C3B681A717B689B88103B5A425341D9
S1134EF0DBB21A1C3B685A71BD4602B080BDC04685
S1134F0084AB0000B0BB0000FCAB0000B4AB0000FD
S1134F1020AC000080B582B000AF7860FB1C197033
S1134F20BB1C1A707B68042B06D9144892235900C1
S1134F30134A144BFDF798FABB1C1B78012B07D9B5
S1134F400E482A23191CFF310D4A0F4BFDF78CFA2A
S1134F50BB1C1B78012B07D17A68FB1C1B78101C27
S1134F60191CFFF71DFF06E07A68FB1C1B78101C58
S1134F70191CFFF7FDFEBD4602B080BD84AB0000E6
S1134F80CCBB0000E0AC0000F4AC000080B582B003
S1134F9000AF7860FB1C1970BB1C1A707B68042B73
S1134FA006D91448A0235900134A144BFDF75CFAA0
S1134FB0BB1C1B78012B06D90E48A22359000E4AAC
S1134FC00F4BFDF751FABB1C1B78012B07D17A68F4
S1134FD0FB1C1B78101C191CFFF7CAFE06E07A683C
S1134FE0FB1C1B78101C191CFFF7DAFEBD4602B02F
S1134FF080BDC04684AB0000E8BB0000E0AC00000C
S1135000F4AC000080B588B000AF786039607B688C
S1135010012B06D92348AD235900234A234BFDF71E
S113502023FA3B68002B07D11E485C23191CFF316F
S11350301D4A1F4BFDF718FA3B681A683B1C0C33DA
S11350401A603B685A683B1C0C335A603B689A6888
S11350503B1C0C339A603B68DA683B1C0C33DA6007
S1135060144B7A689200D2583B1C0C33101C191C48
S113507003F036FF031CFB61FA69AF23DB009A429D
S113508001D10D4B0AE0FB69002B01D1002305E09F
S1135090FB69042B01D1042300E0084B181CBD4616
S11350A008B080BD84AB000008BC0000A4AB0000C5
S11350B014AD000074BB00007427000075270000C5
S11350C080B582B000AF78607B68181C02F07CFA6F
S11350D0031C181CBD4602B080BDC04680B582B01A
S11350E000AF786039607A683B68101C191C02F0C4
S11350F087FABD4602B080BD80B582B000AF78604B
S113510039607B681A683B681A437B681A60BD463D
S113511002B080BD80B582B000AF00237B600A4B33
S1135120181CFFF7CDFF031C7B60074B181C2021C4
S1135130FFF7D4FF7A682023134002D0034B0122E7
S11351401A70BD4602B080BD80F00F4094E0FF1F8E
S113515080B582B000AF00237B60124B181CFFF7B0
S1135160AFFF031C7B600F4A7B68101C191CFFF700
S1135170B5FF7A6880235B01134002D00A4B0122F9
S11351801A707A681023134002D0084B01221A7057
S11351907A682023134002D0054B01221A70BD46C1
S11351A002B080BD00F00F4096E0FF1F97E0FF1FA4
S11351B098E0FF1F80B500AF044B181C8021FFF757
S11351C09BFF034B01221A70BD4680BD00000440C2
S11351D095E0FF1F80B582B000AF786039607B68CE
S11351E03A685A60BD4602B080BDC04680B582B000
S11351F000AF786039607B683A689A60BD4602B057
S113520080BDC04680B582B000AF786039607B68ED
S11352103A68DA60BD4602B080BDC04680B582B04F
S113522000AF786039607A683B68101C191CFFF77E
S1135230E9FFBD4602B080BD80B582B000AF7860A2
S11352400A1CFB1C1A707B68FA1C12781A70BD4683
S113525002B080BD80B584B000AF78607B681B6805
S1135260FB60FB6880229343FB60FB68012293434D
S1135270FB607B68FA681A60BD4604B080BDC04616
S113528080B500AF174B1B78DBB2002B03D0164B55
S1135290181CFDF72BF9154B1B78DBB2002B03D040
S11352A0134B181CFDF722F9124B1B78DBB2002BB1
S11352B003D0114B181CFDF719F9104B1B78DBB206
S11352C0002B03D00E4B181CFDF710F90D4B1B7867
S11352D0DBB2002B03D00C4B181CFDF707F9BD46BD
S11352E080BDC04694E0FF1F70AD000095E0FF1F35
S11352F088AD000096E0FF1FACAD000097E0FF1FF3
S1135300BCAD000098E0FF1FCCAD000080B500AF3D
S1135310084B00221A70084B00221A70074B002217
S11353201A70074B00221A70064B00221A70BD46F1
S113533080BDC04694E0FF1F95E0FF1F96E0FF1F6D
S113534097E0FF1F98E0FF1F80B582B000AF0023F5
S11353507B6000233B6001F031FE031C181C1E21FE
S1135360FBF72EF9031C3B6000237B6002E07B68A3
S113537001337B607A683B689A42F8D3034A8023FE
S11353801B06101C191CFFF749FFEDE700F10F4045
S113539080B584B000AF78603B1C0B3300221A70D8
S11353A00023FB60164B1A683B1C0B33101C191CA2
S11353B000F08AFE031CFB603B1C0B331B785BB2C2
S11353C0104A101C191CFDF791F83B1C0B331B7879
S11353D05AB27B680120111C1A1C00F091F8FB687A
S11353E0002B08D1084B1A687B68101C191CFEF7A7
S11353F083FB031CFB60FB68181CBD4604B080BD26
S11354009CE0FF1FDCAD0000A8E0FF1F90B585B055
S113541000AF78603B1C0E3300221A800023BB606F
S1135420154B1B683C1C0E34144A101C00211A1C1A
S1135430FFF726FC031C23803B1C0E331B88104AF9
S1135440101C191CFDF752F83B1C0E331A887B689C
S11354500320111C1A1C00F053F80A4B1A687B68CD
S1135460101C191CFEF748FB031CBB60BB68181C0E
S1135470BD4605B090BDC046A0E0FF1F00B003408C
S1135480F8AD0000A8E0FF1F80B584B000AF7860DD
S11354903B1C0A3300221A800023FB60154B1A6858
S11354A03B1C0A33101C191C00F07EFE031CFB601D
S11354B03B1C0A331B88104A101C191CFDF716F8F4
S11354C03B1C0A331B881A1C7B680220111C1A1C03
S11354D000F016F8094B1A687B68101C191CFEF7BB
S11354E00BFB031CFA681343FB60FB68181CBD46E6
S11354F004B080BDA4E0FF1F10AE0000A8E0FF1FB1
S113550080B584B000AFB9607A603B1C0F33021CD5
S11355101A707B685B683A1C0F3212781A707B68C9
S11355205B680133BA68120ED2B21A707B685B688A
S11355300233BA68120CD2B21A707B685B68033308
S1135540BA68120AD2B21A707B685B680433BA680C
S1135550D2B21A70BD4604B080BDC04680B586B0D4
S113556000AF01237B613B1D05221A703B1D3A1CD1
S11355700C325A603B1C0C33181C0021052204F029
S1135580F6FC3B1D181CFFF703FF031C7B617B69C2
S1135590002B05D13B1D181CFFF738FF031C7B6152
S11355A07B69002B05D13B1D181CFFF76DFF031C05
S11355B07B617B69181CBD4606B080BDB0B586B062
S11355C002AF78600023FB603B1C0B3300221A708F
S11355D0494B181CFCF78AFF484B1B78DBB2002BA5
S11355E008D0474B181CFCF781FF3B1C0B330022EF
S11355F01A7028E0434B1B78DBB2002B08D0424BD7
S1135600181CFCF773FF3B1C0B3301221A701AE0C1
S11356103E4B1B78DBB2002B08D03D4B181CFCF72B
S113562065FF3B1C0B3302221A700CE0394B1B78CC
S1135630DBB2002B07D0384B181CFCF757FF3B1C80
S11356400B3303221A702D4B1B78DBB2002B0ED1C7
S11356502C4B1B78DBB2002B09D12C4B1B78DBB213
S1135660002B04D12B4B1B78DBB2002B1FD02B4B10
S113567018687B689A787B68DB7879680D79796833
S11356804C79391C0B31097800950194FEF716FB0F
S1135690031CFB60214B1A683B1C0B331B78101C4A
S11356A0191CFEF795FB031CFA681343FB601C4BA3
S11356B01B78DBB2002B13D1104B1B78DBB2002B11
S11356C00ED1104B1B78DBB2002B09D10F4B1B788A
S11356D0DBB2002B04D10F4B1B78DBB2002B06D0BE
S11356E0FB68002B03D1FFF739FF031CFB60FB6849
S11356F0181CBD4604B0B0BD28AE000096E0FF1FE4
S113570058AE000097E0FF1F6CAE000098E0FF1F4A
S113571080AE000094E0FF1F94AE0000A8E0FF1FDD
S113572095E0FF1FB0B586B002AF78600023FB6040
S11357307B681B7801225340DBB2002B19D0002078
S113574004F01CF9FB68002B0CD11F4B1B68181CC0
S1135750FEF78EF9031CFB60FB68002B02D17B680B
S113576001221A70FB68002B03D1184B181CFCF79C
S1135770BDFE7B685B78002B20D0FB68002B1DD11D
S1135780114B18687B6859787B689A787B68DB785A
S11357907C6825797C68647900950194FEF78EFA1B
S11357A0031CFB60084B1A687B685B78101C191C8F
S11357B0FEF70EFB031CFA681343FB60FB68181C1E
S11357C0BD4604B0B0BDC046A8E0FF1FA8AE0000AF
S11357D080B584B000AF78600023FB607B681B78E1
S11357E0002B12D0FB68002B06D10E4B1B68181C33
S11357F0FEF764F9031CFB60FB68002B05D17B6892
S113580000221A70012004F0B9F8FB68002B03D1C0
S1135810054B181CFCF76AFEFB68181CBD4604B057
S113582080BDC046A8E0FF1FD0AE000080B500AF29
S1135830012001F07BF80023181CBD4680BDC04642
S113584080B582B000AF00237B600B4B1B68181C33
S113585000F082FC031C7B6072B6FFF757FD62B652
S1135860064A80231B06101C191CFFF7B3FC7B6837
S1135870181CBD4602B080BDA4E0FF1F00F10F401C
S113588080B500AFE123DB00181C01F04FF8054B95
S1135890181CFCF72BFE01F091F80023181CBD46E0
S11358A080BDC046F8AE000080B584B000AF78601B
S11358B00023FB603F4A80231B06101C191CFFF7C2
S11358C095FCFFF7DDFC3C4B181CFFF7C3FC3B4B7E
S11358D01B78DBB21A1C3A4B1B78DBB21A43394BE8
S11358E01B78DBB21A43384B1B78DBB21A43374BB5
S11358F01B78DBB21343012B05D17B68181CFFF71F
S113590011FF031CFB60FB68002B1BD12B4B1B7886
S1135910DBB21A1C2A4B1B78DBB21A43294B1B78C7
S1135920DBB21A43284B1B78DBB21A43274B1B7894
S1135930DBB21343012B05D17B68181CFFF73EFE35
S1135940031CFB60FB68002B05D17B68181CFFF768
S11359503FFF031CFB601A4B1B78DBB2002B06D005
S1135960144A80231B06101C191CFFF733FC72B663
S11359703B1C0B33114A12781A70FFF7C7FC62B64E
S1135980FB68002B10D13B1C0B331B78002B0BD076
S11359900F4B1B68181C00F0DFFB031CFB60FB684B
S11359A0002B01D0FB6800E0FB68181CBD4604B066
S11359B080BDC04600F10F400000044094E0FF1F8A
S11359C095E0FF1F96E0FF1F97E0FF1F98E0FF1F81
S11359D0A4E0FF1F80B584B000AF78600123FB60B2
S11359E0184B1B78DBB21A1C174B1B78DBB21A431B
S11359F0164B1B78DBB21A43154B1B78DBB21343EF
S1135A00012B09D17B6800229A717B68181CFFF76F
S1135A104BFF031CFB6010E00E4B1B78DBB2002B2A
S1135A2009D07B6802229A717B68181CFFF73CFF3F
S1135A30031CFB6001E00123FB60FB68181CBD46EE
S1135A4004B080BD94E0FF1F96E0FF1F97E0FF1FA6
S1135A5098E0FF1F95E0FF1F80B584B000AF786029
S1135A600023FB607B689B79012B10D002DC002BA8
S1135A7005D043E0022B1BD0032B21D03EE0FFF7DF
S1135A80D5FE031CFB607B6801229A7138E01F4B32
S1135A901B78DBB2002B0AD01C4B00221A70FFF7D4
S1135AA0CFFE031CFB607B6802229A7128E027E08A
S1135AB0FFF7E6FE031CFB607B6803229A711FE07C
S1135AC0134B1B78DBB21A1C104B1B78DBB21A4346
S1135AD0104B1B78DBB21A430F4B1B78DBB21A4313
S1135AE00E4B1B78DBB21343012B06D17B68181CC9
S1135AF0FFF770FF031CFB6002E001E00123FB6081
S1135B00FB68181CBD4604B080BDC04695E0FF1F6D
S1135B1094E0FF1F96E0FF1F97E0FF1F98E0FF1F30
S1135B2080B584B000AF78600023FB607B680022FE
S1135B305A707B6800229A707B680022DA707B6856
S1135B4001221A717B6800225A717B6801221A7043
S1135B507B6800229A7172B6FFF7D8FB62B605E043
S1135B607B68181CFFF778FF031CFB60FB68002BA5
S1135B70F6D0FB68181CBD4604B080BDF0B591B0EA
S1135B8004AF78600023FB627B68002B05D13448A6
S1135B903449354A354BFCF767FC3B1C243300225F
S1135BA05A603B1C243300221A703B1C1C333A1CE1
S1135BB00C325A603B1C1C330F221A7079683A1C51
S1135BC024323B1C1C330F200090081C0D21FDF7D0
S1135BD091FD031CFB62FB6A002B3CD13B1C1C3374
S1135BE01B780F2B02D0224BFB6234E03B1C1C338E
S1135BF05B6808331B78191C3B1C1C335B68093336
S1135C001B781A1C3B1C1C335B680A331B781C1C56
S1135C103B1C1C335B680B331B789C463B1C1C33BE
S1135C205B680C331B781E1C3B1C1C335B680D33F8
S1135C301B781D1C3B1C1C335B680E331B78181C23
S1135C400C4B3B60634600930196029503903868C1
S1135C50231CFCF74BFCFB6A181CBD460DB0F0BDC1
S1135C6014AF00008603000020BC000028AF000031
S1135C70252C000044AF000080B5BCB002AF7860B2
S1135C800123E422D21913603B1C103300221A6052
S1135C9000225A603B1C0833CB221A703B1C083389
S1135CA03A1C18325A603B1CE33300221A7079689C
S1135CB03A1C10323B1C0833CB200090081C0821EE
S1135CC0FDF718FD031CE422D21913603B1C0833B2
S1135CD01B78172B03D00123E422D2191360E4228A
S1135CE0D2191368002B00D08BE03B1CE333002255
S1135CF01A70474B181CFCF7F9FB3B1CE3331B7869
S1135D0003333A1C1832D35C1A1C3B1CE3331B7854
S1135D100233391C1831CB5C3E49081C111C1A1C77
S1135D20FCF7E4FB3B1CE3331B7801333A1C1832C9
S1135D30D35C1A1C3B1CE3331B78391C1831CB5C35
S1135D403549081C111C1A1CFCF7D0FB3B1CE3331F
S1135D5004221A70314B181CFCF7C8FB3B1CE333BC
S1135D601B783A1C1832D35C1A1C3B1CE3331B7897
S1135D700133391C1831CB5C2649081C111C1A1C30
S1135D80FCF7B4FB3B1CE3331B7802333A1C183298
S1135D90D35C1A1C3B1CE3331B780333391C1831C6
S1135DA0CB5C1C49081C111C1A1CFCF79FFB3B1CF8
S1135DB0E3331B7804333A1C1832D35C1A1C3B1CA3
S1135DC0E3331B780533391C1831CB5C1149081CAB
S1135DD0111C1A1CFCF78AFB3B1CE3331B780633AB
S1135DE03A1C1832D35C1A1C3B1CE3331B78073370
S1135DF0391C1831CB5C0849081C111C1A1CFCF70F
S1135E0075FBE422D2191368181CBD463AB080BD54
S1135E105CAF00006CAF000078AF000084AF0000FE
S1135E2080B592B000AF00237B643B1C3C3300225E
S1135E301A6000225A603B1C343300221A6000228C
S1135E405A603B1C2C3300221A6000225A603B1D0E
S1135E5000221A6000229A8000229A71484B3A1C50
S1135E603C321A60474B3A1C34321A60464B3A1C97
S1135E702C321A60454B3A1C0C321A60444B181CE5
S1135E802A21FFF7D9F903F077FC03F0B5FB03F0FF
S1135E908BFB00F0A5FD031C7B647B6C002B05D001
S1135EA03C4A7B6C101C191CFCF720FB3A4A8023EB
S1135EB01B06101C191CFFF799F97B6C002B14D1DD
S1135EC0381C3C30391C2C313A1C34323B1C0C330A
S1135ED000F0EAFC031C7B647B6C002B05D02F4A8A
S1135EE07B6C101C191CFCF701FB7B6C002B26D16E
S1135EF02B4AE123DB00101C191CFCF7F7FA294B91
S1135F00181CFCF7F3FA3B1C0C33181CFFF736FE85
S1135F10031C7B64244B181CFCF7E8FA234B181C65
S1135F20FCF7E4FA3B1C0C33181CFFF7A5FE031C1A
S1135F307A6C13437B641D4B181CFCF7D7FA7B6CFB
S1135F40002B15D1144A80231B06101C191CFFF7C3
S1135F5041F93B1D181CFFF7E3FD031C7B647B6CBC
S1135F60002B05D0124A7B6C101C191CFCF7BEFADE
S1135F70FFF7EAF90023181CBD4612B080BDC046E5
S1135F809CE0FF1FA0E0FF1FA4E0FF1FA8E0FF1F8D
S1135F9000E0074090AF000000F10F40C8AF0000E0
S1135FA000B0000090B20000A4B20000A8B200004B
S1135FB0E8B2000080B584B000AF78600023FB60D5
S1135FC07B681B881BB27A68128812B25343FB6049
S1135FD07B685B881BB27A68528812B25343FA68B2
S1135FE0D318FB607B689B881BB27A68928812B2D4
S1135FF05343FA68D318FB60FB68181CBD4604B011
S113600080BDC04680B588B000AF786039603B1C65
S1136010133300221A700023BB613B1C0C33002293
S11360201A6000229A8000237B613B6800221A6078
S11360307A683B1C1333101C00211A1C0123FEF741
S113604093F9031CBA691343BB613B1C13331A78DD
S11360503F231340DAB23B1C13331A703B1C1F332B
S113606000221A7023E07A683B1C0C33101C191CA4
S1136070FEF7BEFA031CBB61BB69002B01D0BB69F0
S11360801EE03B1C0C33181CFFF794FF031C7B61C0
S11360903B681A687B699A4202D23B687A691A6043
S11360A03B1C1F331A783B1C1F3301321A703B1CF4
S11360B013331B783A1C1F3212789A42D3D300232D
S11360C0181CBD4608B080BD80B586B000AF7860AE
S11360D0396000237B613B1C0D3300221A707B68FE
S11360E0181CFEF787FC031C7B617B69002B01D025
S11360F07B692DE07A683B1C0D33101C191CFEF7DC
S113610089FC031C7B617B69002B01D07B691FE048
S11361103B1C0D331B7801225340DBB2002BE9D129
S11361207868391C12313A1C10323B1C0E33FEF7CE
S113613097FC031C7A6913437B617A683B68101CE3
S1136140191CFEF7CDFC031C7A6913437B617B6940
S1136150181CBD4606B080BD80B584B000AF786021
S11361600023FB603B1C0B3300221A707A683B1C33
S11361700B33101C1E211A1C0123FEF7F5F8031C17
S1136180FB607A683B1C0B33101C00211A1C012392
S1136190FEF7EAF8031CFA681343FB60FB68181C5B
S11361A0BD4604B080BDC04690B585B000AF7860F0
S11361B039600023FB600023BB607A683B1C083312
S11361C0101C191CFFF71EFF031CFB60BB68181C86
S11361D0FAF706FB031C181CFCF7D6F8031C0C1C6E
S11361E0181C211C03F000FD031C0C1C181C211C92
S11361F0FAF7D6FA031C9AB23B681A80FB68181C9B
S1136200BD4605B090BDC04680B582B000AF021C4B
S1136210FB1D1A70FB1D1B787F2B0AD8064BFA1D39
S11362201278111C1F220A400121081C9040021CF4
S11362301A60BD4602B080BD00E100E080B582B0C6
S113624000AF021CFB1D1A70FB1D1B785BB21A1CED
S1136250803201D1012306E0FB1D1B785BB2181CC0
S1136260FFF7D2FF0023181CBD4602B080BDC04614
S113627080B582B000AF78600A1CFB1C1A70FB1C4E
S11362801B78002B06D07B681B6A40221A437B686C
S11362901A6207E07B681B6A4022191C91430A1C9E
S11362A07B681A62BD4602B080BDC04680B584B02A
S11362B000AFF860B960FB1D1A70FB68BA68920001
S11362C0D258084B1A40FB1D1B781902E023DB004F
S11362D00B40111C1943FB68BA689200D150BD46AB
S11362E004B080BDFFF8FFFF80B584B000AF7860D4
S11362F039607B681B68FB60FB6880229343FB600A
S1136300FA683B681343FB607B68FA681A60BD4611
S113631004B080BD80B582B000AF786039607B681E
S11363201A683B681A437B681A60BD4602B080BD98
S113633080B582B000AF786039603B68002B07D12C
S113634007483E23191CFF31064A074BFCF78CF81B
S11363503B685A1E7B689A60BD4602B080BDC04649
S11363601CB3000044BC000034B3000080B584B00A
S113637000AF78607B681B68FB60FB6880229343F6
S1136380FB60FB6801221343FB607B68FA681A60B8
S1136390BD4604B080BDC04680B584B000AF78600F
S11363A07B681B68FB60FB6880229343FB60FB688F
S11363B001229343FB607B68FA681A60BD4604B00F
S11363C080BDC04680B582B000AF78607B68DB7862
S11363D0DBB2181CBD4602B080BDC04690B585B086
S11363E000AF0A1CFB1D011C1970BB1D1A703C1C5C
S11363F00F340F4B181CFFF7E5FF031C2370BB1D64
S11364001B78012B09D0BB1D1B78042B05D0094B2D
S1136410181C01210222FFF749FF3B1C0F331B7894
S1136420042B01D103F0C0F8BD4605B090BDC046B1
S113643000E007400090044080B582B000AF0A1C21
S1136440FB1D011C1970BB1D1A70C0460D4B181C96
S113645002F0EEF8021C8023DB031340F6D0FCF7B5
S11364603DF8BB1D1B78012B09D0BB1D1B78042BE9
S113647005D0054B181C01210022FFF717FFBD466C
S113648002B080BD004005400090044080B584B057
S113649000AF0023FB603B1C181C01F019FA3B1CE5
S11364A0084A5A60002000F09FFD031CFB60064967
S11364B03A1CFB68081C111C1A1C01F07BF9BD4630
S11364C004B080BDA08601000060064080B584B0A1
S11364D000AF78603B1C08330E4A1A603B1C08333B
S11364E00E221A713B1C083301229A713B1C08339B
S11364F000225A713B1C08331422DA717A683B1C5F
S11365000833101C191CFEF727F9031C181CBD4680
S113651004B080BD0060064080B586B000AF7860EE
S11365203B1C083300221A6000225A6000221A72AF
S113653000237B613B1C0833181C00F055FB3B1CFB
S1136540083303221A713B1C083301221A70114AC2
S11365503B1C0833101C191C00F0B6FA0D4B181C18
S11365600021FFF785FE0B4B181C00F06FFB031C8A
S11365707A6913437B617B6803221A607B6800227B
S11365801A717B6800225A717B69181CBD4606B0DB
S113659080BDC04600B0034080B582B000AF3B1D53
S11365A000221A803B1D00225A703B1D01221A70E2
S11365B0294A3B1D101C1F211A1C00F0C9FF1E2074
S11365C0FFF73CFE3B1D00225A703B1D00221A704F
S11365D0224A3B1D101C0C211A1C00F0B9FF1F4A53
S11365E03B1D101C04211A1C00F0B2FF1B4A3B1D6A
S11365F0101C05211A1C00F0ABFF1F20FFF71EFE24
S11366003B1D00225A703B1D00221A70144A3B1D88
S1136610101C05211A1C00F09BFF3B1D00225A7020
S11366203B1D01221A700F4A3B1D101C05211A1C28
S113663000F08EFF0B4A3B1D101C06211A1C00F0B3
S113664087FF084A3B1D101C07211A1C00F080FF1D
S1136650BD4602B080BDC04600F10F4000F00F40BF
S113666080F00F40C0F00F4080B588B000AF786074
S11366700023FB613B1C0833384A1A603B1C083377
S11366801D221A713B1C083301225A713B1C08332A
S11366900122DA713B1C083330229A713B1C1433FB
S11366A00E221A703B1C143301221A713B1C143342
S11366B001225A703B1C1433FA22D2005A803B1C2C
S11366C01033C0221A703B1C103320229A703B1CDA
S11366D0103300225A707A683B1C0833101C191CB2
S11366E0FDF702FD031CFA691343FB617B68181C68
S11366F00021FDF749FF031CFA691343FB617A6823
S11367003B1C1433101C191CFDF74EFD031CFA69C5
S11367101343FB617A683B1C1033101C191CFDF7F2
S1136720A5FD031CFA691343FB617B68181C052152
S11367300122FDF7D9FE031CFA691343FB617B6850
S1136740181C0121FDF720FF031CFA691343FB61A8
S1136750FB69181CBD4608B080BDC04600600640F9
S113676090B585B000AF021CBB1D1A80BB1D1C88F0
S1136770132000F039FC031C1A1C6243274B9A4275
S113678006D92748A8235900264A274BFBF76CFE55
S1136790BB1D1C88132000F027FC031C63437F2BC4
S11367A007D81F485223191CFF311E4A1F4BFBF701
S11367B05BFE3B1C0833181C01F0E4FC3B1C083353
S11367C006229A713B1C083300221A71184A3B1C9A
S11367D00833101C191C01F085FC154B181CFFF71D
S11367E0DBFDBB1D1C88132000F0FEFB031C634370
S11367F0DB090F4A101C191CFFF79AFD0C4B181CDF
S11368008021FFF787FD0A4B181C4021FFF76CFD20
S11368101C20FFF713FDBD4605B090BD7FFF7F0030
S113682040B3000038BC000054B3000084B300003F
S11368300000044080B584B000AF78603B1C08338E
S1136840181CFCF731FF7B6803221A737B68022251
S11368501A617B6803221A757B6804229A617B683B
S11368600C33181CFDF7C6FB7B680E4A9A600020A7
S113687000F0BAFB021C7B685A607B6801221A6034
S11368807B68181C0021FDF76DFB7A683B1C0833FC
S1136890101C191CFCF782FE031C181CBD4604B016
S11368A080BDC046A086010080B586B000AFF86008
S11368B0B9607A603B6000237B61FFF7E7FDFFF777
S11368C06BFEFB68181CFFF701FE031C7B617B69F0
S11368D0002B01D07B6924E07B68181CFFF71CFEA9
S11368E0031C7B617B69002B01D07B6919E03B6849
S11368F0181CFFF79FFF031C7B617B69002B01D0F1
S11369007B690EE0BB68181CFFF7AEFE031C7B61BD
S11369107B69002B01D07B6903E00120FFF720FF96
S11369207B69181CBD4606B080BDC04680B582B0E8
S113693000AF7860132000F057FB031C7A685A43B9
S1136940184B9A4206D91848DB235900174A184BAA
S1136950FBF78AFD132000F047FB031C7A685343BE
S11369607F2B07D81048B823191CFF310F4A114B4D
S1136970FBF77AFD104B181CFFF70EFD132000F0F7
S113698033FB031C7A685343DB090B4A101C191CA4
S1136990FFF7CEFC084B181CFFF7E8FCBD4602B01D
S11369A080BDC0467FFF7F0040B300005CBC000098
S11369B054B3000084B300000000044080B500AF6D
S11369C004201021FFF738FD044B181C01F0C4FF0C
S11369D004201021FFF702FDBD4680BD00E0074002
S11369E080B582B000AF00233B60002000F0FCFAC9
S11369F0031C7B60114B181C01F08AFF031C3B60D5
S1136A003B68002B01D03B6813E002E07B68013B4C
S1136A107B600A4B181CFFF7D5FC031C042B02D027
S1136A207B68002BF2D17B68002B01D1052300E0A9
S1136A300023181CBD4602B080BDC04600E00740DC
S1136A4090B585B000AF78607B681B0C084A9B1832
S1136A50FB60FB68FA6811687A681204120C012062
S1136A60041C9440221C0A431A60BD4605B090BD24
S1136A700070044080B584B000AF78600023FB60F0
S1136A8007E00D4A7B689A4200D105E0FB680133B8
S1136A90FB60FB68002BF4D0FB68002B06D0074991
S1136AA0074A084B081C4A21FBF7DEFCFB68181C4C
S1136AB0BD4604B080BDC04600B00340ACB3000086
S1136AC074BC0000C4B3000080B584B000AF78602B
S1136AD039603B68002B06D13F49404A404B081CB3
S1136AE05121FBF7C1FC7B68181CFFF7C3FF3D4B2A
S1136AF0181CFFF7A5FF3B685B781A1C03231A4098
S1136B003B681B7999000C230B401343FB603B68E3
S1136B105B79042B03D0FB6810221343FB603B68B2
S1136B20DB785A0160231340FA681343FB603B6827
S1136B30DB79002B03D0FB6880221343FB607B6866
S1136B40FA689A607B68DB680F229343FB603B68BA
S1136B505B79042B07D03B685B791A1C0323134031
S1136B60FA681343FB603B689B79002B03D0FB68F6
S1136B7004221343FB603B689B78002B03D0FB6823
S1136B8008221343FB607B68FA68DA607B681B6A3F
S1136B9003229343FB603B681B781A1C03231340B6
S1136BA0FA681343FB607B68FA681A623B681B7AD5
S1136BB0002B06D07B685B6A08221A437B685A6202
S1136BC007E07B685B6A0822191C91430A1C7B68F6
S1136BD05A62BD4604B080BDACB3000088BC00005E
S1136BE0E8B300001B003C1080B582B000AF7860B1
S1136BF07B68002B06D11249124A134B081C9121C1
S1136C00FBF732FC7B6800221A707B6803225A70FF
S1136C107B6801229A707B680322DA707B68012208
S1136C201A717B6804225A717B6800229A717B680E
S1136C300022DA717B6800221A72BD4602B080BD60
S1136C40ACB3000094BC0000E8B3000080B586B08B
S1136C5000AF78603B1C173300221A7000233B619D
S1136C607B681A6A402313400BD03B1C1733012264
S1136C701A707B681B6A4022191C91430A1C7B68AA
S1136C801A627B685B6AC0221A437B685A620AE014
S1136C907B68181C00F068F8021C4023134002D0E3
S1136CA001233B6108E07B68181C002100F0BAF85E
S1136CB0021C80231340EBD07B681B69FB603B1CE8
S1136CC017331B78002B05D07B681B6A40221A43BC
S1136CD07B681A627B68181C00F046F8021C40238B
S1136CE0134001D001233B613B69002B01D03B6978
S1136CF036E07B68DA6C7B689B6CD2187B685B6CD3
S1136D00D2187B681B6CD2187B68DB6BD2187B684B
S1136D109B6BD318FB60FB685B0880221202134351
S1136D20FB60FA687B68DA627B68DA6E7B689B6E6C
S1136D30D2187B685B6ED2187B681B6ED2187B6896
S1136D40DB6DD2187B689B6DD318FB60FB685B0816
S1136D50802212021343FB60FA687B681A630023E3
S1136D60181CBD4606B080BD80B584B000AF786005
S1136D700023FB607B681A6A8023134003D0FB68FE
S1136D8080221343FB607B685A6A4023134003D07C
S1136D90FB6840221343FB60FB68181CBD4604B02B
S1136DA080BDC04680B586B000AFF860B9607A6037
S1136DB0BB68012B07D917485823191CFF31164A01
S1136DC0164BFBF751FB7B68002B06D11148AC2313
S1136DD05900114A124BFBF747FB7B681A681F23C3
S1136DE013407B617B685B79002B03D07B69202295
S1136DF013437B617B681B79002B03D07B694022A2
S1136E0013437B61FB68BA6892007969D150BD462F
S1136E1006B080BDACB30000ACBC0000F8B3000009
S1136E20E8B3000080B584B000AF786039603B6897
S1136E30012B07D90C486E23191CFF310B4A0C4B4C
S1136E40FBF712FB0023FB607B683A689200D25880
S1136E508023134003D0FB6880221343FB60FB684C
S1136E60181CBD4604B080BDACB30000C4BC000017
S1136E70F8B3000080B582B000AF7860074B074AD2
S1136E801168074A11407A689004C0221203024034
S1136E900A431A60BD4602B080BDC046007004407B
S1136EA0FFFFF3FF80B500AF0E4B1B78DBB21A1C5B
S1136EB00223134008D10B4B9B79DBB21A1C0C2321
S1136EC013409B08012B09D1064B5B78DBB21A1CDB
S1136ED001231A40044B9200D35800E00023181CED
S1136EE0BD4680BD0040064030BD000080B500AF07
S1136EF00C4B1B78DBB2DBB25BB2002B0DDA0A4B16
S1136F001B68002B06D10949094A0A4B081C892130
S1136F10FBF7AAFA044B1B6800E00023181CBD46CB
S1136F2080BDC0460050064010E1FF1F18B40000A9
S1136F3038BD000030B4000080B582B000AF1A4BF9
S1136F401A68C0231B0313409B0C022B10D0032B85
S1136F501DD0002B1FD1FFF7C9FF021C80231B0289
S1136F609A4202D180231B0200E000237B6015E0DB
S1136F700E4B1B68002B06D10D490E4A0E4B081C04
S1136F809D21FBF771FA094B1B687B6006E0FA232D
S1136F909B007B6002E000237B60C0467B68181C7A
S1136FA0BD4602B080BDC046007004400CE1FF1F26
S1136FB018B4000050BD00003CB4000080B500AF20
S1136FC000F0CAF8021C0649064BCB581B0F0133CC
S1136FD0101C191CF9F7F4FA031C181CBD4680BDDB
S1136FE0007004404410000080B584B000AF021C5F
S1136FF0FB1D1A70FB1D1B78132B48D89A00284BD5
S1137000D3181B689F4600F0A7F8021C2549264B9D
S1137010CB581B0F0133101C191CF9F7D1FA031CB0
S1137020FB6037E000F098F8021C1E491E4BCB5859
S11370301B0F0133101C191CF9F7C2FA031CFB6067
S1137040184A194BD258E023DB0213401B0C0133BE
S1137050F868191CF9F7B4FA031CFB601AE0FFF78F
S11370606BFF031CFB6015E0FFF740FF031CFB6094
S113707010E000F031F8031CFB600BE000F050F866
S1137080031CFB6006E0FA239B00FB6002E0002384
S1137090FB60C046FB68181CBD4604B080BDC046FA
S11370A0E0BC0000007004404410000080B582B0D1
S11370B000AF7860064A7B685968064BD1507B68FC
S11370C01B78181CFFF7D6FEBD4602B080BDC04633
S11370D0007004404410000080B582B000AF0F4B34
S11370E01B7ADBB21A1C0E2313405A08FB1D1A70BC
S11370F00A4B1B7ED9B2BB1D07220A401A70FFF748
S1137100D1FE021CFB1D1978BB1D1B78CB18111C6A
S1137110D9400B1C181CBD4602B080BD004006407F
S113712080B500AF0A4B1B7EDBB2DBB25BB2002B37
S113713007DB074B9B79DBB21A1C0C2313409B081B
S113714001D1044B00E00023181CBD4680BDC0469D
S113715000400640006CDC0280B582B000AF1B4BDF
S11371609B79DBB21A1C0C2313409B08012B06D01D
S113717002D3022B12D020E0154B7B6020E0FFF7F6
S113718091FE021C114B1B7ADBB2191C0E230B401F
S11371905B08111CD9400B1C7B6011E00D4B1B6874
S11371A0002B06D10C48992359000C4A0C4BFBF7D1
S11371B05BF9084B1B687B6002E000237B60C046E0
S11371C07B68181CBD4602B080BDC0460040064026
S11371D0006CDC0210E1FF1F18B4000068BD000061
S11371E030B4000080B582B000AF78607B68002BBB
S11371F007D142485E23191CFF31414A414BFBF73A
S113720033F9414B9B79DBB21A1C0C2313409B08C6
S1137210012B1ED17B681B78012B1AD13A4B5B786A
S1137220DBB21A1C01231A407B689B789A4210D067
S1137230354B354A1278D1B23F220A40D2B21A7085
S1137240C046314B9B79DBB21A1C0C2313409B08BC
S1137250F7D12D4A7B68DB78DB18D9B20E230B40BB
S1137260DBB21372284B7A685279D201D1B27A68B0
S1137270107907220240D2B20A43D2B21A76224BC4
S1137280214A5278D2B201218A43D1B27A689078E5
S113729001220240D2B20A43D2B25A701A4B7A681F
S11372A012789201D1B27A6852780A43D2B21A7033
S11372B0154B5B78DBB21A1C042313400BD07B689C
S11372C01B78022B07D1C0460F4B9B79DBB21A1CEB
S11372D002231340F8D0C0467B681B781A1C0A4B63
S11372E09B79DBB2191C0C230B409B089A42F3D107
S11372F00023181CBD4602B080BDC04618B400006F
S11373007CBD00004CB400000040064080B584B051
S113731000AFF860B9607A60BB68032B07D91048E6
S1137320DE23191CFF310F4A0F4BFBF79DF87B68D6
S1137330002B12D0F968BA6884235B0012018A1802
S1137340D3181B68802252041A43F868B96884234E
S11373505B0009014118CB181A60BD4604B080BD1A
S11373605CB40000A4BD000074B4000080B582B019
S113737000AF78607B68002B07D111482223191CC9
S1137380FF31104A104BFBF76FF87B6819687B6874
S11373901B791A1C80235B04081C111C1A1CFFF7A0
S11373A0B5FF7B689B68002B07D07B689A687B6875
S11373B0DB687968081C191C9047BD4602B080BD83
S11373C0A0B4000094BD000018B5000080B500AF63
S11373D0034B1B68181CFFF7C9FFBD4680BDC046A0
S11373E0ACE0FF1F80B500AF034B5B68181CFFF7D0
S11373F0BDFFBD4680BDC046ACE0FF1F80B500AFF9
S1137400034B9B68181CFFF7B1FFBD4680BDC04607
S1137410ACE0FF1F80B500AF034BDB68181CFFF71F
S1137420A5FFBD4680BDC046ACE0FF1F80B582B05D
S113743000AFFB1D00221A701DE0FB1D1A78114BD2
S11374409200D358002B11D0FB1D1A780E4B9200DA
S1137450D358FA1D11780D4A89008958FA1D1078FD
S1137460084A80008258081C111C9847FB1D1A7892
S1137470FB1D01321A70FB1D1B78012BDDD9BD46A3
S113748002B080BDBCE0FF1FCCE0FF1FC4E0FF1FC3
S113749080B500AFFFF7CAFFBD4680BD80B584B09C
S11374A000AFF860B960FB1D1A70FB1D1B78002B40
S11374B005D1BB6801229A40FB689A6004E0BB686E
S11374C001229A40FB685A60BD4604B080BDC046A4
S11374D080B584B000AFF860B960FB1D1A70F9681C
S11374E0BA68FB1D1B78081C111C1A1CFFF7D6FF79
S11374F0BD4604B080BDC04680B584B000AF78609E
S11375000023FB600AE00E4BFA689200D2587B68B5
S11375109A4200D105E0FB680133FB60FB68042B51
S1137520F1D9FB68042B06D90649074A074B081C06
S11375305821FAF799FFFB68181CBD4604B080BDBA
S1137540D4BD0000C4B50000E8BD0000DCB50000F7
S113755080B584B000AFF860B9607A607B68002BB6
S113756006D11649164A174B081C5F21FAF77CFF0F
S11375707B681B78002B0BD1FB685B69BA6801211F
S1137580081C9040021CD2431A40FB685A6112E066
S11375907B685B78F968BA68081C111C1A1CFFF731
S11375A097FFFB685A69BB680121081C9840031CBB
S11375B01A43FB685A61BD4604B080BDC4B50000DF
S11375C0FCBD000000B6000080B584B000AF786058
S11375D07B68181CFFF790FF021C3B1C0F331A70CA
S11375E03B1C0F331A78054B9200D358BB60BA6822
S11375F0A023D358181CBD4604B080BDC0BD0000F4
S113760080B584B000AF786039607B68181CFFF7E0
S113761073FF021C3B1C0F331A703B1C0F331A7888
S1137620054B9200D358BB60BA68A0233968D15087
S1137630BD4604B080BDC046C0BD000090B585B055
S113764000AF78607B681B0C084A9B18FB60FB68E2
S1137650FA6811687A681204120C0120041C944020
S1137660221C0A431A60BD4605B090BD0070044058
S113767080B582B000AF786039603A6880235B01DE
S1137680134009D07B689B79DAB23B681B0ADBB2F2
S11376901343DAB27B689A713A688023DB011340A2
S11376A009D07B689B79DAB23B681B0ADBB21343CF
S11376B0DAB27B689A713B68DAB27B68DA70BD46ED
S11376C002B080BD80B584B000AF78600023FB6059
S11376D00AE00E4BFA689200D2587B689A4200D1B5
S11376E005E0FB680133FB60FB68012BF1D9FB6803
S11376F0012B06D90649074A074B081CB921FAF79A
S1137700B3FEFB68181CBD4604B080BD8CBE0000EF
S11377102CB600009CBE000044B6000080B584B0C6
S113772000AF786039600023FB603A68102313408F
S113773005D07B681022DA70064BFB6005E03A68DE
S11377400123134001D0044BFB60FB68181CBD46A9
S113775004B080BD4F0400004E04000080B582B028
S113776000AF786039607B68DB78DBB21A1C1023C9
S1137770134006D17B689B78DBB21A1C202313408C
S113778007D00A4B1B6879683A68081C111C984793
S113779006E0074B1B6879683A68081C111C984777
S11377A0BFF34F8FBD4602B080BDC046DCE0FF1F73
S11377B0E0E0FF1F80B586B000AFF860B9607A6082
S11377C0BB68002B02D07B68002B06D13B48FD230D
S11377D059003B4A3B4BFAF747FEFB68181CFFF77E
S11377E071FF021C384B9200D358181CFFF726FF78
S11377F0FB6800221A70FB6800225A70FB680022A2
S11378009A70FB68FF22DA70FB6800225A71FB68E9
S113781050229A71FB680022DA71FB689B78DAB215
S11378207F231340DAB2FB689A70FA68274B101C66
S1137830191CFFF71DFFBB685A68F9687B68081CB0
S1137840111C1A1C00F06AF83B1C1733FA68927971
S11378501A703B1C17333A1C173211787F220A40E6
S11378601A70BB685B78DB01D9B23B1C17333A1C36
S1137870173212780A431A703B1C17333A1C17321A
S113788012780F218A431A70BB681A7A0F231340A7
S1137890D9B23B1C17333A1C173212780A431A70B8
S11378A0FB683A1C173212789A71BB681B78DB01AB
S11378B0DAB2FB689A70BD4606B080BD2CB60000F3
S11378C0ACBE000068B6000094BE00001250000078
S11378D080B582B000AF78607B68002B05D10A4880
S11378E00A490B4A0B4BFAF7BFFD7B680A4A5A60F8
S11378F07B6800225A707B6800221A727B6801221E
S11379001A70BD4602B080BD2CB6000043020000D0
S1137910BCBE000084B60000A086010080B58CB017
S113792000AFF860B9607A6001235B42FB62002318
S1137930BB6200237B623B1C233300221A704BE0A2
S11379403B1C23331B780122111C99400B1CFB6147
S11379503B1C223300221A7032E03B1C22331A787B
S1137960294B5200D35AFA6953437868191CF8F723
S113797027FE031CBB61BA68BB699A4203D9BA6883
S1137980BB69D31A02E0BA69BB68D31A7B617A690E
S1137990FB6A9A420DD23B1C23331B78BB623B1C0F
S11379A022331B787B627B69FB627B69002B00D1ED
S11379B00BE03B1C22333A1C2232127801321A703B
S11379C03B1C22331B783F2BC7D93B1C23333A1C67
S11379D02332127801321A703B1C23331B78022B9A
S11379E002D8FB6A002BABD1BB6ADBB29B01DAB2D3
S11379F07B6AD9B23F230B40DBB21343DAB2FB6894
S1137A005A70BD460CB080BD0CBE000080B584B079
S1137A1000AF7860FB1C1970BB1C1A700023FB605C
S1137A207B68181C00F0B2F8031CBB60BA68202302
S1137A30134002D0134BFB601EE07B689B78DBB2E3
S1137A4030221343DAB27B689A70C0467B681B7B92
S1137A50DBB21A1C01231340F8D0FB1C1B78DB1883
S1137A60DAB2BB1C1B78012B01D1012300E00023F7
S1137A701343DAB27B681A71FB68181CBD4604B064
S1137A8080BDC0464C04000080B586B000AF78606D
S1137A90FB1C1970BB1C1A7000237B617B68181CCB
S1137AA000F074F8031CFB603B1C133306221A70AD
S1137AB0FA682023134009D07B689B78DBB21A1C38
S1137AC02023134002D1224B7B613BE03B1C0B3350
S1137AD07A6852781A703B1C0B331A783F23134090
S1137AE0DAB27B685A707B689B78DBB2142213434A
S1137AF0DAB27B689A707B683A1C0B3212785A703F
S1137B0000E0C0463B1C13331B783A1C1332591E49
S1137B101170002BF5D1C0467B681B7BDBB21A1CAD
S1137B2001231340F8D0FB1C1B78DB18DAB2BB1C12
S1137B301B78012B01D1012300E000231343DAB2A7
S1137B407B681A717B69181CBD4606B080BDC046AF
S1137B504C04000080B584B000AF78600023FB6063
S1137B607B689B78DBB238229343DAB27B689A70E5
S1137B70C0467B68DB78DBB21A1C20231340F8D1A3
S1137B80FB68181CBD4604B080BDC04680B584B0F7
S1137B9000AF78607B68DB78DBB2FB607B689B7945
S1137BA0DBB21A1C4023134004D0FB688022D201AC
S1137BB01343FB607B689B79DBB21A1C10231340D0
S1137BC004D0FB68802252011343FB60FB68181C3D
S1137BD0BD4604B080BDC04680B586B000AFF86035
S1137BE0B9607A603B6000237B613B1C1333002245
S1137BF01A70C046FB68DB78DBB2DBB25BB2002BE9
S1137C00F8DAFB680222DA70FB689B78DBB2102298
S1137C101343DAB2FB689A7032E0BB685A1CBA604C
S1137C201A78FB681A71C046FB68DB78DBB21A1C51
S1137C3002231340F8D03B1C1333FA68D2781A702D
S1137C40FB680222DA703B1C13331A7810231340AA
S1137C5004D0FB681022DA70184B7B613B1C133391
S1137C601A780123134007D07B68002B04D0FB68EB
S1137C700122DA70124B7B617B69002B00D004E097
S1137C807B685A1E7A60002BC7D17B69002B03D115
S1137C903A680423134003D07A69094B9A4208D105
S1137CA0FB680222DA70FB68181CFFF753FF031C01
S1137CB07B617B69181CBD4606B080BD4F04000083
S1137CC04E04000080B586B000AFF860B9607A60F9
S1137CD03B6000237B613B1C133300221A703B1C66
S1137CE013331B78DBB20133DAB23B1C13331A7043
S1137CF0C046FB68DB78DBB2DBB25BB2002BF8DAA0
S1137D00FB680222DA70FB689B78DBB2182293438B
S1137D10DAB2FB689A707B68012B07D1FB689B7809
S1137D20DBB208221343DAB2FB689A70FB681B7952
S1137D30DAB23B1C13331A7032E0C046FB68DB78BE
S1137D40DBB21A1C02231340F8D0FB680222DA705B
S1137D507B68002B12D13A680423134006D1FB68D8
S1137D60181CFFF7F7FE031C7B6107E0FB689B7898
S1137D70DBB210221343DAB2FB689A707B68012BE2
S1137D8007D1FB689B78DBB208221343DAB2FB68A5
S1137D909A70BB685A1CBA60FA681279D2B21A7027
S1137DA07B685A1E7A60002BC7D17B69181CBD46BC
S1137DB006B080BD80B584B000AF786039603B68A0
S1137DC0002B06D18F488023D9008F4A8F4BFAF7B6
S1137DD04BFB3B1C0F333A6852791A700023BB608B
S1137DE07A688B4B101C191CFFF742FCC0467B6859
S1137DF0DB78DBB2DBB25BB2002BF8DA3B681B7BCF
S1137E00002B07D03B685B79012B03D13B1C0F335C
S1137E1000221A703B681A680123134006D03B1CE9
S1137E200F331B78012B21D10423E7E03B681A6848
S1137E30022313400DD03B681A7979683B1C0F3339
S1137E401B78081C111C1A1CFFF71EFE031CBB60C8
S1137E500CE03B681A7979683B1C0F331B78081CCB
S1137E60111C1A1CFFF7D2FD031CBB603B681A6887
S1137E700123134025D1BB68002B01D0BB68BDE0B2
S1137E80C0467B68DB78DBB21A1C02231340F8D0AF
S1137E907B68DB78DBB27A68101C191CFFF73EFCA8
S1137EA0031CBB60BB68002B0BD0BA68594B9A42C9
S1137EB005D1594BBB607B68181CFFF74BFEBB68B0
S1137EC09CE03B681B7B002B00D170E07B680222A6
S1137ED0DA703B681B7B013BDAB23B681A733B6880
S1137EE09A683B681B7BDB00111CD9400B1CDAB27F
S1137EF07B681A71C0467B68DB78DBB21A1C0223EC
S1137F001340F8D07B68DB78DBB27A68101C191C4C
S1137F10FFF704FC031CBB60BB68002B09D0BA68E4
S1137F203C4B9A4203D17B68181CFFF713FEBB68D5
S1137F3064E03B681B7B002B02D0BB68002BC5D0E0
S1137F403B685B79012B32D17B680222DA703B6893
S1137F501B797A68101C191C0122FFF795FD031C7C
S1137F60BB60BB68002B01D0BB6847E0C0467B68A0
S1137F70DB78DBB21A1C02231340F8D07B68DB7871
S1137F80DBB27A68101C191CFFF7C8FB031CBB602A
S1137F90BB68002B0BD0BA681E4B9A4205D11E4B0E
S1137FA0BB607B68181CFFF7D5FDBB6826E03B6807
S1137FB05B79002B0ED13B685B69002B0AD03B68D0
S1137FC019693B685A693B681B687868FFF704FEC7
S1137FD0031CBB603B685B79012B0ED13B685B697A
S1137FE0002B0AD03B6819693B685A693B681B68D7
S1137FF07868FFF767FE031CBB60BB68181CBD46AE
S113800004B080BD2CB60000D8BE000094B60000B9
S1138010125000004E0400005104000080B500AF6F
S1138020044B1B68044A101C191CFFF797FBBD4640
S113803080BDC046D4E0FF1F0060064080B500AF9D
S1138040044B5B68044A101C191CFFF787FBBD46F0
S113805080BDC046D4E0FF1F0070064090B585B0D7
S113806000AF78607B681B0C084A9B18FB60FB68B8
S1138070FA6811687A681204120C0120041C9440F6
S1138080221C0A431A60BD4605B090BD007004402E
S113809080B584B000AF78600023FB6007E00D4A30
S11380A07B689A4200D105E0FB680133FB60FB6802
S11380B0002BF4D0FB68002B06D00749074A084B75
S11380C0081C5721FAF7D0F9FB68181CBD4604B008
S11380D080BDC04600000440F4B60000F4BE0000B9
S11380E00CB7000080B584B000AF786039603B689D
S11380F0002B06D11F49204A204B081C5F21FAF7A8
S1138100B3F97B68181CFFF7C3FF031CFB601C4B0F
S1138110181CFFF7A3FF3B681B785A0002231A4080
S11381203B68DB78990004230B401A433B689B7837
S1138130D90008230B401A433B685B7819013023AC
S11381400B401A437B681A603B689B79DA007823FA
S11381501A403B681B79990004230B401A433B687F
S11381605B79191C03230B401A437B685A60BD4694
S113817004B080BDF4B6000008BF000030B70000B2
S11381800000381080B582B000AF78607B68002BA7
S113819006D10F490F4A104B081C8E21FAF764F9D7
S11381A07B6800221A707B6800225A707B68002268
S11381B09A707B680022DA707B6801221A717B68EE
S11381C001225A717B6800229A71BD4602B080BDBB
S11381D0F4B6000014BF000030B7000090B585B0BD
S11381E000AF78607B681B0C084A9B18FB60FB6837
S11381F0FA6811687A681204120C0120041C944075
S1138200221C0A431A60BD4605B090BD00700440AC
S113821090B585B000AF78607B681B0C094A9B1849
S1138220FB60FB68FA68126879680904090C01208C
S1138230041C8C40211CC9430A401A60BD4605B089
S113824090BDC0460070044080B584B000AF786033
S11382500023FB600AE00E4BFA689200D2587B6858
S11382609A4200D105E0FB680133FB60FB68012BF7
S1138270F1D9FB68012B06D90649074A074B081CAC
S11382809021FAF7F1F8FB68181CBD4604B080BDD4
S11382902CBF000038B700003CBF000050B70000FE
S11382A090B58DB000AFF860B9607A60BB68002B00
S11382B006D19F499F4AA04B081CE721FAF7D4F83E
S11382C0BB681B68002B06D199499A4A9B4B081C32
S11382D0E821FAF7C9F8BB681B68BB6100237B621D
S11382E03B1C2A3300221A8004233B625DE0BB68F6
S11382F01B683A6A53437868191CF8F761F9031C40
S11383001A1C3B1C28331A803B1C28331B88002B67
S113831003D13B1C283301221A803B1C28331B88C1
S11383203A6A53437868191CF8F74AF9031C7B61CD
S1138330BB681B687A69D31AFB61BB681C683B1C69
S113834028331B8801333A6A53437868191CF8F7B9
S113835037F9031CE21AFB699A4215D2BB681C6800
S11383603B1C28331B8801333A6A53437868191C31
S1138370F8F726F9031CE31AFB613B1C28331A881F
S11383803B1C283301321A80FA69BB699A4209D826
S1138390FB69BB613B6A7B623B1C2A333A1C283273
S11383A012881A803B6A01333B623B6A202B9ED9B8
S11383B0BB681B68181C6421F8F702F9031C1A1C1B
S11383C0131C5B009A18BB699A4201D25C4BABE068
S11383D0FB68181CFFF738FF031C3B61594B3A69D3
S11383E09200D358181CFFF7F9FEFB689A68564BA5
S11383F01A40FB689A60FB681B68FB627B6A032B6C
S113840007D97B6A072B04D8FB6A802292021343A4
S1138410FB62FA6A4D4B1340FB627B6A013B1A060E
S1138420F8235B051340FA6A1343FB62FB6A5B0B98
S11384305B03FB623B1C2A331B88DB04DA0CFB6AFC
S11384401A43FB681A60FB681A68414B1A40FB68C0
S11384501A60FB689A683F4B1340FB62BB681B7948
S11384601A1CBB685B7A1902E023DB000B401A4339
S1138470BB681B7A990004230B401343FA6A134325
S1138480FB62BB681B79002B03D0FB6A10221343E9
S1138490FB62FB68FA6A9A60FB681A682E4B134009
S11384A0FB62BB68DB795A0380239B011A40FB6A99
S11384B01A43FB681A60294BFB62FB6A802212068E
S11384C01343FB62FB6AC02212021343FB62BB68C4
S11384D09B79002B05D0FB6A802292051343FB6233
S11384E003E0FA6A1A4B1340FB62FB685A68FB6AA2
S11384F01A43FB685A60FB689B68FB62BB689B7A03
S1138500002B04D0FB6A802212031343FB62BB6876
S1138510DB7A002B04D0FB6A8022D2021343FB6275
S1138520FB68FA6A9A600023181CBD460DB090BD22
S113853038B7000050BF000088B7000090B70000B3
S11385402105000034BF0000FFFFF3FFFFFFFFE041
S1138550FFFFFFDFE8F8FFFFFFDFFFFF00001F4022
S113856080B584B000AF7860C0467B685A688023C9
S1138570DB031340F9D0124BFB60FB688022120628
S11385801343FB60FB68C02212021343FB607B6849
S11385905A68FB681A437B685A607B6800229A60B9
S11385A07B68181CFFF750FE031CBB60054BBA68C0
S11385B09200D358181CFFF72BFEBD4604B080BDB3
S11385C000001F4034BF000080B582B000AF786067
S11385D07B68002B07D11348E623191CFF31124A8C
S11385E0124BF9F741FF7B68E12252021A607B6863
S11385F000221A717B6800225A717B6800229A71EA
S11386007B680022DA717B6800221A727B68002280
S11386105A727B6800229A727B680022DA72BD4625
S113862002B080BD38B700005CBF000088B700000E
S113863080B584B000AF78607B685B68FB60FB68E2
S1138640181CBD4604B080BD80B584B000AF78600E
S113865039607B685B68BB60BB685B005B08BB60C0
S11386603B68DB0FDB07BA681343BB60BA68144B83
S11386701340BB603A68134B1340BA681343BB60A2
S1138680BA68114B1340BB603A68C0231B02134005
S1138690BA681343BB607B68BA685A607B68181C6D
S11386A0FFF7C6FF031C3A68134002D0074BFB6078
S11386B001E00023FB60FB68181CBD4604B080BDCC
S11386C0FFFFE0BF00001F40FF3FFFFF1A0500004F
S11386D080B584B000AFF860B9607A60BB68002BE5
S11386E006D10F48AB2399000E4A0F4BF9F7BCFE95
S11386F00DE0C046FB685A6880231B041340F9D080
S1138700BB685A1CBA601B781A1CFB68DA607B6869
S11387105A1E7A60002BECD1BD4604B080BDC04621
S113872038B7000074BF000080B7000080B586B081
S113873000AFF860B9607A60BB68002B05D12F48A0
S11387402F49304A304BF9F78FFE4CE03EE0FB688E
S1138750181CFFF76DFF031C7B617A6980231B03E0
S1138760134008D0FA6880231B03101C191CFFF760
S11387706BFF264B3DE07A698023DB02134008D06F
S1138780FA688023DB02101C191CFFF75DFF204BE5
S11387902FE07A6980239B02134008D0FA68802373
S11387A09B02101C191CFFF74FFF1A4B21E07A693A
S11387B080235B02134009D0FA6880235B02101CFB
S11387C0191CFFF741FFA423DB0012E0FB685A6881
S11387D080239B031340BAD0BB685A1CBA60FA6862
S11387E0D268D2B21A707B685A1E7A60002BADD15F
S11387F00023181CBD4606B080BDC04638B7000033
S1138800BB0200008CBF000080B700001D05000003
S11388101E0500001F05000080B500AF044B1A6858
S1138820044B1B680449081C191C9047BD4680BDB5
S1138830ECE0FF1FE4E0FF1F0040054080B500AFFF
S1138840044B1A68044B5B680449081C191C9047C4
S1138850BD4680BDECE0FF1FE4E0FF1F0050054073
S113886080B500AF264B5B68002B23D0254A8023BC
S1138870D25880239B02134006D1224A8023D25827
S11388808023DB02134015D01E4A8023D258802354
S11388909B00134006D11B4A8023D2588023DB005F
S11388A0134007D0184B1A68154B5B681549081C10
S11388B0191C9047124B1B68002B1FD0114B1A68D0
S11388C080239B02134005D10E4B1A688023DB02E0
S11388D0134013D00B4B1A6880239B00134005D11F
S11388E0084B1A688023DB00134007D0074B1A6833
S11388F0034B1B680349081C191C9047BD4680BDE7
S113890014E1FF1F00F00240F4E0FF1FF0E0FF1F3E
S113891080B584B000AF78603B1C0F337A6852781E
S11389201A703B1C0F333A1C0F32127860218A43B1
S11389301A703B1C0F333A1C0F32127840210A4341
S11389401A707B683A1C0F3212785A700023181C74
S1138950BD4604B080BDC04680B584B000AF786029
S11389603B1C0F337A6852781A703B1C0F333A1C45
S11389700F32127807218A431A703B1C0F333A1CBA
S11389800F32127802210A431A707B683A1C0F32A4
S113899012785A700D4B0D4A126904210A431A6168
S11389A07B685B78BFF34F8F30BFBFF36F8F7B68FB
S11389B05B78DBB21A1C0823134001D0044B00E09F
S11389C00023181CBD4604B080BDC04600ED00E085
S11389D03C0F000090B585B000AF78607B681B0C3D
S11389E0084A9B18FB60FB68FA6811687A681204ED
S11389F0120C0120041C9440221C0A431A60BD4638
S1138A0005B090BD0070044080B584B000AF7860BC
S1138A100023FB600AE00E4BFA689200D2587B6890
S1138A209A4200D105E0FB680133FB60FB68012B2F
S1138A30F1D9FB68012B06D90649074A074B081CE4
S1138A409921F9F711FDFB68181CBD4604B080BDDF
S1138A50A0BF0000F0B70000B0BF000008B80000DD
S1138A6080B584B000AF78600A1CFB1C1A707B6868
S1138A70181CFFF7C9FF031CFB60044AFB68D318EA
S1138A80FA1C12781A70BD4604B080BD08E1FF1FBD
S1138A9080B588B000AFF860B9607A600023FB61EC
S1138AA03B1C1B3301221A70FB68181CFFF7ACFF38
S1138AB0031C7B61FB689B78DBB21A1C40231340C8
S1138AC09B09DAB23B1C1B3301321A7036E0BB68D7
S1138AD0002B1AD0FB689B78DBB21A1C402313408E
S1138AE00CD0BB685A1CBA601A78FB689A71BB68D0
S1138AF05A1CBA601A78FB68DA7119E0BB685A1C10
S1138B00BA601A78FB689A7112E0104A7B69D3182C
S1138B101B78DBB21B029AB20C497B69CB181B7819
S1138B20DBB213439BB2FA68101C191C00F0A0F9C5
S1138B303B1C1B331B78FA69D318FB61FA697B6809
S1138B409A42C4D3BD4608B080BDC04608E1FF1FA9
S1138B5080B586B000AFF860B9607A6000237B61AD
S1138B603B1C133301221A70FB689B78DBB21A1C7E
S1138B70402313409B09DAB23B1C133301321A70B1
S1138B802AE0BB68002B1DD0FB689B78DBB21A1C63
S1138B90402313400ED0BB685A1CBA60FA6892791D
S1138BA0D2B21A70BB685A1CBA60FA68D279D2B2CF
S1138BB01A700BE0BB685A1CBA60FA689279D2B298
S1138BC01A7003E0FB68181C00F068F93B1C1333AF
S1138BD01B787A69D3187B617A697B689A42D0D30F
S1138BE0BD4606B080BDC04680B582B000AF786097
S1138BF07B6801221A707B6800225A707B6800220D
S1138C009A707B680022DA707B6800221A717B6894
S1138C1000225A717B6801229A717B680122DA7101
S1138C207B6800225A727B6803221A727B68024AAC
S1138C30DA60BD4602B080BD20A1070080B584B0D3
S1138C4000AFF860B9607A60BB68002B02D07B6823
S1138C50002B07D15348AE23191CFF31524A534B02
S1138C60F9F702FCFB68181CFFF7CEFE021C504B00
S1138C709200D358181CFFF7ADFEFB68DB78DBB21B
S1138C8040229343DAB2FB68DA70BB689B78DB005E
S1138C90DAB208231340DAB2BB68DB789B00D9B29E
S1138CA004230B40DBB21343DAB2BB68197A012305
S1138CB00B40DBB2DB18D9B202230B40DBB2134307
S1138CC0DAB2BB68197901230B40DBB21343DBB280
S1138CD010221343DAB2FB68DA70BB681B7A5B08B4
S1138CE0DBB21B01DAB210231340DAB2BB685B7A41
S1138CF05B08DBB2DB00D9B208230B40DBB21343C1
S1138D00DAB2BB685B78DB18D9B202230B40DBB262
S1138D101343DAB2BB68597A01230B40DBB2134325
S1138D20DAB2BB685B799B01D9B240230B40DBB25A
S1138D301343DAB2FB689A70FA681E4B9A4214D055
S1138D40BB689B795B01DAB220231340DAB2BB68BB
S1138D50DB791B01D9B210230B40DBB21343DBB226
S1138D6001221343DAB2FB68DA72BB68DA68F96885
S1138D707B68081C111C1A1C00F01EF8FB68181CE8
S1138D80FF21FFF76DFEBB681B78002B07D0FB6843
S1138D90DB78DBB240221343DAB2FB68DA70BD46FB
S1138DA004B080BDF0B70000C0BF00002CB80000C4
S1138DB0A8BF00000060074080B58EB000AFF86027
S1138DC0B9607A60BB68FB6101235B423B620723A5
S1138DD03B630823BB6200237B632FE002237B6297
S1138DE00023FB6221E07B6B01337A6A534378688A
S1138DF0191CF7F7E5FB031CBB61FA69BB699A42CE
S1138E000DD3FA69BB69D31A7B613A6A7B699A42CA
S1138E1005D97B693B627B6B3B63FB6ABB627B6A04
S1138E205B007B62FB6A0133FB62FB6A082B02D89E
S1138E303B6A002BD7D17B6B01337B637B6B072BA6
S1138E4002D83B6A002BC9D1BB6ADAB20F231340A4
S1138E50DAB23B6BDBB21B01D9B270230B40DBB23D
S1138E601343DAB2FB685A70BD460EB080BDC046EB
S1138E7080B582B000AF78600A1CBB1C1A80BB1C92
S1138E801B88DAB27B689A71BB1C1B881B0A9BB2D5
S1138E90DAB27B68DA71BD4602B080BD80B584B0B9
S1138EA000AF78603B1C0E3300221A807B689B79EC
S1138EB0DAB23B1C0E331A807B68DB79DBB21B020F
S1138EC099B23B1C0E333A1C0E3212880A431A80A4
S1138ED03B1C0E331B88181CBD4604B080BDC04625
S1138EE080B584B000AF786039603B68002B06D150
S1138EF03F48BE2399003F4A3F4BF9F7B5FA3B1C64
S1138F000F3301221A703B681B68002B05D13B68A4
S1138F105B68002B01D1042365E07B689B78DBB29E
S1138F201A1C402313409B09DAB23B1C0F33013255
S1138F301A707A68314B9A4208D07B68DB7ADBB2CC
S1138F4001229343DAB27B68DA7247E046E0C04616
S1138F507B681B78DBB21A1C20231340F8D03B68D3
S1138F601A683B1C0F331B787968081C111C1A1CE7
S1138F70FFF78EFD3B681B68002B08D03B681A681E
S1138F803B1C0F331B78D2183B681A60FFE7C046BE
S1138F907B681B78DBB2DBB25BB2002BF8DA3B6890
S1138FA05A683B1C0F331B787968081C111C1A1C67
S1138FB0FFF7CEFD3B685B68002B07D03B685A681F
S1138FC03B1C0F331B78D2183B685A603B689A6885
S1138FD03B1C0F331B78D21A3B689A603B689B6832
S1138FE0002BB4D10023181CBD4604B080BDC0467C
S1138FF0F0B70000D0BF00004CB80000006007408C
S113900080B582B000AF786039607B68DB78DBB212
S11390101A1C102313400AD00B4B1B680B4A3968E7
S113902089008A587968081C111C984709E0084B84
S11390301B68064A396889008A587968081C111C1B
S11390409847BD4602B080BD00E1FF1FF8E0FF1F56
S113905004E1FF1F80B500AF084B1B68002B05D14E
S113906007480849084A094BF9F7FEF9084B181C48
S11390700021FFF7C5FFBD4680BDC046F8E0FF1FD5
S1139080F0B7000023040000ECBF00006CB800003F
S11390900060074080B500AF084B5B68002B05D12A
S11390A007480849084A094BF9F7DEF9084B181C28
S11390B00121FFF7A5FFBD4680BDC046F8E0FF1FB4
S11390C0F0B700002B04000004C000007CB80000CE
S11390D00070074090B585B000AF78607B681B0CCA
S11390E0084A9B18FB60FB68FA6811687A681204E6
S11390F0120C0120041C9440221C0A431A60BD4631
S113910005B090BD0070044090B585B000AF7860A4
S11391107B681B0C094A9B18FB60FB68FA681268A1
S113912079680904090C0120041C8C40211CC943E2
S11391300A401A60BD4605B090BDC04600700440A8
S113914080B584B000AF78600323BB600023FB606C
S11391500AE00F4BFA689200D2587B689A4200D119
S113916006E0FB680133FB60FA68BB689A42F0D3FF
S1139170FA68BB689A4206D30649074A074B081C9B
S1139180A521F9F771F9FB68181CBD4604B080BD30
S11391901CC000008CB8000034C00000A4B800005B
S11391A080B588B000AFF860B9607A60BB68002B06
S11391B006D18149814A824B081CD021F9F754F920
S11391C0BB681B68002B06D17B497C4A7D4B081C7D
S11391D0D121F9F749F93B1C1E3300221A803B1CAC
S11391E01D3300221A700023BB61BB681B681B017E
S11391F07868191CF7F7E4F9031C1A1C3B1C1E338E
S11392001A803B1C1E331B88002B03D13B1C1E33CE
S113921001221A8000237B617B685A00BB681B68AB
S1139220101C191CF7F7CCF9031C99B23B1C1E3314
S11392301B882022524253439AB23B1C12338A1891
S11392401A807B685A003B1C1E331B8859013B1C47
S113925012331B88CB18101C191CF7F7B1F9031C27
S11392607B61BB681A687B699A4204D2BB681B683D
S11392707A69D31A03E0BB681A687B69D31ABB61A5
S1139280BB681B68181C6421F7F79AF9031C1A1CA5
S1139290131C5B009A18BB699A4201D24A4B87E0BF
S11392A0FB68181CFFF74CFF021C484B9200D35874
S11392B0181CFFF70FFFFB68DB78DBB20C2293432B
S11392C0DAB2FB68DA70FB681B78DBB21F229343C7
S11392D0DAB23B1C1E331B881B0A9BB2DBB213435E
S11392E0DAB2FB681A703B1C1E331B88DAB2FB68C7
S11392F05A70FB689B7ADBB21F229343DAB23B1CA1
S113930012331B88D9B21F230B40DBB21343DAB2EA
S1139310FB689A72FB689B78DAB23B1C1D331721F9
S11393208A431A70BB685B799B00DAB2042313404A
S1139330D9B23B1C1D333A1C1D3212780A431A70F1
S1139340BB681B79002B0BD0BB681A793B1C1D33FF
S11393501B781343DAB23B1C1D3310210A431A70E5
S1139360FB683A1C1D3212789A703B1C1D33FA6854
S1139370D2781A70BB689B79002B07D03B1C1D3335
S11393803A1C1D32127808210A431A70BB68DB7933
S1139390002B07D03B1C1D333A1C1D3212780421CC
S11393A00A431A70FB683A1C1D321278DA700023E3
S11393B0181CBD4608B080BD8CB8000048C0000031
S11393C0C8B80000D0B80000F503000028C00000B1
S11393D080B582B000AF7860C0467B681B79DBB291
S11393E01A1C40231340F8D07B680022DA707B6893
S11393F0181CFFF7A5FE021C044B9200D358181C3E
S1139400FFF782FEBD4602B080BDC04628C0000002
S113941080B582B000AF78607B68002B07D10D481F
S11394207023191CFF310C4A0C4BF9F71DF87B68AB
S1139430E12252021A607B6800221A717B680022C2
S11394405A717B6800229A717B680022DA71BD46EA
S113945002B080BD8CB8000054C00000C8B8000041
S113946080B584B000AF78607B681B79DBB21A1CCE
S11394707B685B79DBB21B021343FB60FB68181C3F
S1139480BD4604B080BDC04680B584B000AFF8606E
S1139490B9607A600DE0C046FB681B79DBB2DBB2D1
S11394A05BB2002BF8DABB685A1CBA601A78FB6806
S11394B0DA717B685A1E7A60002BECD1BD4604B089
S11394C080BDC04680B586B000AFF860B9607A60F0
S11394D0BB68002B05D11F481F49204A204BF8F7D1
S11394E0C3FF2DE01EE0FB68181CFFF7B9FF031C47
S11394F07B617A690823134001D01A4B26E07A690C
S11395000423134001D0184B20E07A69022313404E
S113951001D0164B1AE07A690123134002D0FD23CF
S11395209B0013E0FB681B79DBB21A1C2023134059
S1139530D9D0BB685A1CBA60FA68D279D2B21A7010
S11395407B685A1E7A60002BCCD10023181CBD46C0
S113955006B080BD8CB80000530200006CC000004F
S1139560F8B80000F1030000F2030000F303000068
S113957080B582B000AF7860084A0849084BC958E2
S1139580084B19407B689806C0231B050340194308
S1139590034BD150BD4602B080BDC04600700440AC
S11395A004100000FFFFFFF380B582B000AF03207A
S11395B0FFF7DEFF0C20FDF717FD031C7B60064957
S11395C096239A017B68081C111C0222F8F760FF9D
S11395D0BD4602B080BDC0460040054080B500AF26
S11395E0024A034B0349D150BD4680BD007004407C
S11395F0441000000000031080B500AFFFF7EEFF39
S1139600064B181CFDF7EEFD054B181CFDF74EFD2F
S1139610044B054A1A60BD4680BDC04680C00000A8
S113962088C0000000E0FF1F80841E0090B585B054
S113963000AF78607B681B0C084A9B18FB60FB68D2
S1139640FA6811687A681204120C0120041C944010
S1139650221C0A431A60BD4605B090BD0070044048
S113966080B586B000AFF860B9607A607B68002B83
S113967006D1094884235900084A094BF8F7F4FE37
S1139680BB689B00FA68D3187B617B697A6812888F
S11396901A80BD4606B080BD38B9000090C00000F5
S11396A050B9000080B584B000AFF860B960FB1D0C
S11396B01A70FB68BA689200D258084B1A40FB1D16
S11396C01B781902E023DB000B40111C1943FB68D3
S11396D0BA689200D150BD4604B080BDFFF8FFFFC8
S11396E080B584B000AFF860B960FB1D1A70FB68E8
S11396F0BA689200D258084B1A40FB1D1B78190413
S1139700F0231B030B40111C1943FB68BA68920039
S1139710D150BD4604B080BDFFFFF0FF80B584B0DA
S113972000AFF860B960FB1D1A70FB1D1B78002B9D
S113973005D1BB6801229A40FB689A6004E0BB68CB
S113974001229A40FB685A60BD4604B080BDC04601
S113975080B584B000AFF860B960FB1D1A70F96879
S1139760BA68FB1D1B78081C111C1A1CFFF7D6FFD6
S1139770BD4604B080BDC04680B582B000AF3B1D7D
S113978000221A803B1C00221A803B1D1A780321F8
S11397900A431A703B1C1A7803218A4302210A43A4
S11397A01A706C4B181CFFF741FF6B4B181CFFF72A
S11397B03DFF6A4B181CFFF739FF694B181CFFF774
S11397C035FF684B181C01210222FFF76BFF654B24
S11397D0181C02210222FFF765FF634A6249634BAA
S11397E0CB580721181C8843011C604BD15000F052
S11397F0F9F85F4A3B1D101C18211A1CFFF730FFB3
S11398005B4A3B1D101C19211A1CFFF729FF584BFA
S1139810181C18210522FFF745FF554B181C192168
S11398200522FFF73FFF534A3B1D101C05211A1C5C
S1139830FFF716FF4F4B181C05210122FFF732FFDB
S11398404C4B181C05210A22FFF74AFF484B181CF1
S11398501F210122FFF726FF474A3B1C101C07214A
S11398601A1CFFF7FDFE444B181C07210222FFF7C8
S113987019FF414A3B1D101C06211A1CFFF7F0FE7C
S11398803D4B181C06210222FFF70CFF3A4A3B1CF1
S1139890101C05211A1CFFF7E3FE374B181C052189
S11398A00222FFF7FFFE344A3B1D101C04211A1C40
S11398B0FFF7D6FE304B181C04210122FFF7F2FEFD
S11398C02D4A3B1D101C02211A1CFFF7C9FE2A4B0E
S11398D0181C02210122FFF7E5FE224A3B1D101C41
S11398E00C211A1CFFF7BCFE1E4B181C0C21012274
S11398F0FFF7D8FE1B4B181C0C210A22FFF7F0FEC1
S1139900184A3B1D101C04211A1CFFF7A9FE154B15
S1139910181C04210122FFF7C5FE124B181C042158
S11399200A22FFF7DDFE0F4A3B1D101C05211A1CFD
S1139930FFF796FE0B4B181C05210122FFF7B2FE20
S1139940084B181C05210A22FFF7CAFEBD4602B0C7
S113995080BDC046090038100B0038100C003810C8
S11399600D003810009004400070044010100000F6
S113997000D0044000B0044000C0044080B584B06E
S113998000AF021CFB1D1A703B1C0F3301221A701E
S1139990FB1D1B78002B01D0012300E002233A1C9D
S11399A00F3213700E4A3B1C0F331B78101C052119
S11399B01A1CFFF777FE0A4A3B1C0F331B78101C56
S11399C006211A1CFFF76EFE054A3B1C0F331B7859
S11399D0101C07211A1CFFF765FEBD4604B080BDAC
S11399E000C0044080B582B000AF3B1D00221A8045
S11399F0FB1D00221A70BB1D00221A703B1D1A7831
S1139A0003210A431A703B1D5A7807218A43012116
S1139A100A435A703B1C01221A703B1C01225A70E3
S1139A20614A3B1D101C18211A1CFFF719FE5E4ADF
S1139A303B1D101C19211A1CFFF712FE5B4A3B1C2C
S1139A40101C18211A1CFDF783FD584A3B1C101CDE
S1139A5019211A1CFDF77CFD544B181C19210022F6
S1139A60FFF776FEFB1D00221A702CE04F4B181CEA
S1139A7018210022FFF76CFEBB1D00221A7005E0BE
S1139A80C046BB1D1A78BB1D01321A70BB1D1B7862
S1139A90FF2BF5D1454B181C18210122FFF758FE66
S1139AA0BB1D00221A7005E0C046BB1D1A78BB1D01
S1139AB001321A70BB1D1B78FF2BF5D1FB1D1A78E0
S1139AC0FB1D01321A70FB1D1B78072BCED9374BB7
S1139AD0181C18210022FFF73BFE344B181C1921D7
S1139AE00122FFF735FEBB1D00221A7005E0C046B7
S1139AF0BB1D1A78BB1D01321A70BB1D1B78FF2BCE
S1139B00F5D12A4B181C18210122FFF721FEBB1D99
S1139B1000221A7005E0C046BB1D1A78BB1D013235
S1139B201A70BB1D1B78FF2BF5D1204B181C182174
S1139B300022FFF70DFEBB1D00221A7005E0C0468F
S1139B40BB1D1A78BB1D01321A70BB1D1B78FF2B7D
S1139B50F5D1164B181C19210022FFF7F9FDBB1D86
S1139B6000221A7005E0C046BB1D1A78BB1D0132E5
S1139B701A70BB1D1B78FF2BF5D10C4B181C182138
S1139B800122FFF7E5FDBB1D00221A7005E0C04667
S1139B90BB1D1A78BB1D01321A70BB1D1B78FF2B2D
S1139BA0F5D1BD4602B080BD00D0044000F10F40A5
S1139BB080B500AF0A4B9B78DBB21A1C0823134014
S1139BC007D0074B064A9278D2B208210A43D2B290
S1139BD09A70044A88235B010021D150BD4680BDA0
S1139BE000D0074000700440F0B5474680B48AB006
S1139BF0041C0D1C00F058F8294A0023D356904643
S1139C00061C0F1C01330DD0201C291C00F032F956
S1139C10002807D0201C291C204B1F4AF6F796FD6C
S1139C20002805D1301C391C0AB004BC9046F0BD94
S1139C30012300931B4B049405950193002308937F
S1139C404346029403951C78002C0ED1134B124A00
S1139C5006920793684600F03DF900280FD0089B50
S1139C60002B11D1069E079FDCE70C490A48021C11
S1139C700B1CF7F727F906900791022CEAD100F0A4
S1139C802BF921230360EAE700F026F9089C04601D
S1139C90E8E7C046C046C0460000000000000000DF
S1139CA004E0FF1FA4C00000F0B55F4656464D46D1
S1139CB04446F0B46C4E0D1C371C83B0041C021CCB
S1139CC00B1C2F40B74200D1ADE0002900DC8BE033
S1139CD02F1500D194E0654D09038023090B5B0324
S1139CE07F190B43FE0700D570E07F10C20FB84602
S1139CF05B00002780219B18162442000097002057
S1139D00890345189D4204DC68185B1B009D6D188F
S1139D100095D50F5B00013C5B1952004908002CEB
S1139D20EFD180210026090620250196B4468946F4
S1139D3009E0834246D0D40F5B00013D1B19520059
S1139D404908002D1CD066468C198342F1DD671842
S1139D50E60FBC46F60782464E452CD01B1AA2429B
S1139D6080414042019F1B1A121B7F18D40F5B00D5
S1139D70013D019750461B1952004908002DE2D1BC
S1139D80134328D101984308009D394E6A10921953
S1139D90ED0702D5802109060B4340460705B91893
S1139DA01C1C0D1C201C291C03B03CBC904699466D
S1139DB0A246AB46F0BDFF0FFF077E427E41B2468E
S1139DC08244CBE79442C2D9181CB4E7C20F5B00AB
S1139DD09B18400089E7019901312FD0019C012390
S1139DE023401B195B08CFE76B005B081A43D9D0EB
S1139DF0002700292BD1C10A153F40050029FAD0BC
S1139E008022520311421ED1002349000133114222
S1139E10FBD001242022E41AD21A3F19041CD44096
S1139E202143984057E7201C291CF7F7B5FC221C56
S1139E302B1CF6F725FD041C0D1CB3E7009A002328
S1139E4001320092A0E7202201240023E5E7221C2E
S1139E502B1C201C291CF7F72FFF021C0B1CF7F7E7
S1139E6031F8041C0D1C9DE70000F07F01FCFFFF8E
S1139E700000E03F0B1C011C021C30B519430220FA
S1139E80002900D130BD802109068B4216D00D492E
S1139E9004205C180C498C42F4D90C4D5C198C429A
S1139EA0F0D90B4C590049080320A142EAD9074CC8
S1139EB00020A142E6D150425041E3E7002AE1D01C
S1139EC0EFE7C0460000F0FFFFFFDF7F0000F07FF8
S1139ED0FFFF0F0000207047014B18687047C04611
S1139EE068E0FF1F084B10B5041C002B02D00021B2
S1139EF000E000BF054B1868836A002B00D0984728
S1139F00201C00F043F8C04600000000B0C0000070
S1139F1070B50E4B0E4D0024ED1AAD101E1CAC4254
S1139F2004D0A300F35898470134F8E702F0C2F8CC
S1139F30084B094D0024ED1AAD101E1CAC4204D090
S1139F40A300F35898470134F8E770BDD4C000006B
S1139F50D4C00000D4C00000D8C0000010B5002355
S1139F60934203D0CC5CC4540133F9E710BD031C05
S1139F708218934202D019700133FAE77047002324
S1139F80C25C0133002AFBD1581E7047FEE7C0466D
S1139F90415353455254204552524F5220222025BA
S1139FA07320223A2066696C652022257322204C96
S1139FB0696E6520222564222066756E6374696F5C
S1139FC06E206E616D652022257322200A00000038
S1139FD02E2E2F7574696C69746965732F66736CA2
S1139FE05F64656275675F636F6E736F6C652E6324
S1139FF00000000064657669636520213D204445C6
S113A0004255475F434F4E534F4C455F4445564975
S113A01043455F545950455F4E4F4E450000000084
S113A0202E2E2F7574696C69746965732F66736C51
S113A0305F696F2E630000004E554C4C20213D207B
S113A040696F00002E2E2F7574696C6974696573CD
S113A0502F66736C5F6C6F672E63000062756620F9
S113A060213D204E554C4C00636820213D204E5527
S113A0704C4C00002E2E2F736F757263652F736620
S113A0802F73662E6300000028636D64203E3D201C
S113A0903078303155292026262028636D64203CF1
S113A0A03D20307832365529000000007061796C0B
S113A0B06F61644C656E203C3D2030784339550017
S113A0C06672616D6520213D202828766F696420C1
S113A0D02A293029000000006472764461746120EA
S113A0E0213D202828766F6964202A293029000020
S113A0F0616D6C5370694461746120213D2028288E
S113A100766F6964202A293029000000616D6C5340
S113A1107069446174612D3E6461746153697A6548
S113A120203E2030550000004750494F5F414D4CC0
S113A1305F52656164496E70757428647276446117
S113A14074612D3E6770696F436F6E6669672E6335
S113A1507350696E2E6770696F496E7374616E63B4
S113A160652C20647276446174612D3E6770696F5A
S113A170436F6E6669672E637350696E2E677069EC
S113A1806F50696E4E756D6265722920213D2030D5
S113A190550000004750494F5F414D4C5F52656187
S113A1A064496E70757428637350696E2D3E6770D0
S113A1B0696F496E7374616E63652C2063735069B3
S113A1C06E2D3E6770696F50696E4E756D62657273
S113A1D02920213D203055006770696F50696E2039
S113A1E0213D202828766F6964202A29302900001F
S113A1F028746D6F75745573203E203055292026C0
S113A200262028746D6F75745573203C20313030CE
S113A21030303030303055290000000073656E64F2
S113A2204C656E203E2030550000000073656E645E
S113A23042756666657220213D202828766F696420
S113A240202A29302900000072656376427566660B
S113A250657220213D202828766F6964202A2930E0
S113A26029000000300000002866726571487A20D9
S113A2703E3D2037373530303030303055292026B8
S113A28026202866726571487A203C3D20313030A2
S113A2903030303030303055290000002828766FB7
S113A2A06964202A29302920213D206672616D6568
S113A2B0000000002828766F6964202A29302920AC
S113A2C0213D206663696E74000000002828766FC3
S113A2D06964202A29302920213D20666366726141
S113A2E06300000073706952637642756620213DF5
S113A2F0202828766F6964202A293029000000006C
S113A300726563765061796C6F616420213D202809
S113A31028766F6964202A29302900002872656331
S113A320765061796C6F61642D3E7061796C6F61F8
S113A330642920213D202828766F6964202A293049
S113A34029000000287366537069436D6453657473
S113A350556C46726571203D3D20636D6429207CF7
S113A3607C20287366537069436D64536574446C30
S113A37046726571203D3D20636D64290000000034
S113A38066726571487A20213D202828766F6964B9
S113A390202A29302900000075736572436F6E66A8
S113A3A0696720213D202828766F6964202A293096
S113A3B02900000073656E645061796C6F616420DC
S113A3C0213D202828766F6964202A29302900003D
S113A3D073656E645061796C6F61642D3E70617950
S113A3E06C6F61644C656E203C3D20307843395578
S113A3F00000000028282828636D6429203D3D20A2
S113A4007366537069436D6453656E644563686F26
S113A41029207C7C202828636D6429203D3D2073FD
S113A42066537069436D6453656E645061796C6FF3
S113A430616429207C7C202828636D6429203D3DAB
S113A440207366537069436D6453656E6442697426
S113A45029207C7C202828636D6429203D3D2073BD
S113A46066537069436D64536574556C46726571C7
S113A47029207C7C202828636D6429203D3D20739D
S113A48066537069436D64436F6E745761766529D2
S113A490207C7C202828636D6429203D3D20736640
S113A4A0537069436D6453656E64546573744D6F82
S113A4B0646529207C7C202828636D6429203D3D27
S113A4C0207366537069436D6450736B41736B5AA8
S113A4D065726F53657129207C7C202828636D6424
S113A4E029203D3D207366537069436D6450736B3E
S113A4F041736B4141414153657129207C7C202883
S113A50028636D6429203D3D207366537069436D53
S113A510645365744643434D6163726F43682920F5
S113A5207C7C202828636D6429203D3D207366537C
S113A5307069436D645374617469634672657143F1
S113A540616C29207C7C202828636D6429203D3D92
S113A550207366537069436D6454656D704672650B
S113A5607143616C29207C7C202828636D64292038
S113A5703D3D207366537069436D6452656365693C
S113A580766529207C7C202828636D6429203D3D44
S113A590207366537069436D64536574446C4672EA
S113A5A065712929202626202873656E64506179F7
S113A5B06C6F61642D3E7061796C6F616420213D24
S113A5C0202828766F6964202A2930292929207CAB
S113A5D07C2028282828636D6429203D3D2073664B
S113A5E0537069436D6453656E644563686F2920D5
S113A5F07C7C202828636D6429203D3D20736653AC
S113A6007069436D6453656E645061796C6F616405
S113A61029207C7C202828636D6429203D3D2073FB
S113A62066537069436D6453656E6442697429208E
S113A6307C7C202828636D6429203D3D207366536B
S113A6407069436D64536574556C46726571292055
S113A6507C7C202828636D6429203D3D207366534B
S113A6607069436D64436F6E745761766529207C0D
S113A6707C202828636D6429203D3D207366537037
S113A68069436D6453656E64546573744D6F64659A
S113A69029207C7C202828636D6429203D3D20737B
S113A6A066537069436D6450736B41736B5A657282
S113A6B06F53657129207C7C202828636D642920D0
S113A6C03D3D207366537069436D6450736B4173F1
S113A6D06B4141414153657129207C7C20282863CA
S113A6E06D6429203D3D207366537069436D645346
S113A6F065744643434D6163726F436829207C7CD3
S113A700202828636D6429203D3D207366537069B9
S113A710436D645374617469634672657143616C1B
S113A72029207C7C202828636D6429203D3D2073EA
S113A73066537069436D6454656D70467265714308
S113A740616C29207C7C202828636D6429203D3D90
S113A750207366537069436D6452656365697665F9
S113A76029207C7C202828636D6429203D3D2073AA
S113A77066537069436D64536574446C46726571C5
S113A7802929203D3D203029000000002873656EF2
S113A790645061796C6F61642D3E7061796C6F6196
S113A7A0644C656E203E20305529202626202873CF
S113A7B0656E645061796C6F61642D3E7061796C73
S113A7C06F616420213D202828766F6964202A293E
S113A7D030292900283055203D3D20626974566196
S113A7E06C29207C7C20283155203D3D20626974F1
S113A7F056616C2900000000646576496E666F201E
S113A800213D202828766F6964202A2930290000F8
S113A810646576496E666F2D3E6C69625665727327
S113A820696F6E20213D202828766F6964202A29CB
S113A830302900007375636365737320213D2028FC
S113A84028766F6964202A293029000028706179EC
S113A8506C6F61644C656E203E203055292026269D
S113A86020287061796C6F61644C656E203C3D20DA
S113A870307830355529000001020304050000003A
S113A8802873664E65745374616E646172644554D2
S113A8905349203C3D207374616E64617264536556
S113A8A06C29202626202873664E65745374616EC5
S113A8B0646172644643435F536F757468416D65A8
S113A8C072696361203E3D207374616E64617264D9
S113A8D053656C29000000002873665874616C3558
S113A8E03532203C3D207874616C292026262028AE
S113A8F073665874616C323736203E3D207874613B
S113A9006C2900002873665478526570656174314F
S113A910203C3D2074785265706561742920262698
S113A92020287366547852657065617433203E3D07
S113A930207478526570656174290000287366502C
S113A940613134203C3D20706154797065292026A2
S113A9502620287366506130203E3D207061547972
S113A9607065290072657065746974696F6E73200F
S113A9703C3D2028696E7431365F74293078464630
S113A980550000002828766F6964202A2930292080
S113A990213D2066684D61736B0000002828766FA6
S113A9A06964202A29302920213D206368616E6E64
S113A9B0656C55736167650031303030303030304C
S113A9C0303055203E3D206472696674487A000038
S113A9D02828766F6964202A29302920213D2064A3
S113A9E0726966745461626C650000002828766F91
S113A9F06964202A29302920213D20647269667403
S113AA005461626C6552657300000000727373696F
S113AA1052657320213D202828766F6964202A29F5
S113AA203029000070615461626C6520213D20284A
S113AA3028766F6964202A2930290000286E6574FD
S113AA40537464203D3D2073664E65745374616E87
S113AA50646172644554534929207C7C20286E65C6
S113AA6074537464203D3D2073664E657453746161
S113AA706E646172644643435F536F757468416DDD
S113AA80657269636129207C7C20286E6574537427
S113AA9064203D3D2073664E65745374616E646139
S113AAA072644643435F55534129207C7C20286EC1
S113AAB06574537464203D3D2073664E657453740D
S113AAC0616E646172644152494229007265637621
S113AAD05061796C6F61642D3E7061796C6F616453
S113AAE020213D202828766F6964202A29302900F6
S113AAF02E2E2F736F757263652F73662F73665FC7
S113AB0073657475702E63006770696F436F6E664A
S113AB10696700002E2E2F736F757263652F6D6D3C
S113AB206138343531712F6D6D612E630000000082
S113AB306669666F436F6E662D3E77617465726DEC
S113AB4061726B436E74203C3D203332550000002B
S113AB502E2E2F647269766572732F66736C5F6133
S113AB60646331362E6800006368616E6E656C47FD
S113AB70726F7570203C204144435F525F434F55D0
S113AB804E5400002E2E2F736F757263652F616D06
S113AB906C2F7370695F616D6C2F7370695F616D89
S113ABA06C2E6300696E7374616E6365203C2028AB
S113ABB03229000073706953646B4D61737465725C
S113ABC0436F6E66696720213D202828766F69648B
S113ABD0202A29302900000073706953646B536C78
S113ABE0617665436F6E66696720213D202828766B
S113ABF06F6964202A2930290000000073706941BC
S113AC006D6C4D6173746572436F6E666967202164
S113AC103D202828766F6964202A29302900000005
S113AC2028737069416D6C4D6173746572436F6E06
S113AC306669672D3E626974436F756E74203D3D8D
S113AC4020385529207C7C2028737069416D6C4D17
S113AC506173746572436F6E6669672D3E626974D1
S113AC60436F756E74203D3D203136552900000038
S113AC70737069416D6C536C617665436F6E666980
S113AC806720213D202828766F6964202A293029ED
S113AC900000000028737069416D6C536C61766527
S113ACA0436F6E6669672D3E626974436F756E7497
S113ACB0203D3D20385529207C7C20287370694133
S113ACC06D6C536C617665436F6E6669672D3E6289
S113ACD06974436F756E74203D3D203136552900EB
S113ACE0706F7274496E7374616E6365203C2028C2
S113ACF035290000706373506F6C61726974792038
S113AD003C3D207370695063734163746976654C8C
S113AD106F7700006D61737465725472616E73664F
S113AD20657220213D202828766F6964202A293005
S113AD3029000000736C6176655472616E736665F8
S113AD407220213D202828766F6964202A29302921
S113AD5000000000736C61766548616E646C652068
S113AD60213D202828766F6964202A293029000093
S113AD70416363656C65726174696F6E20646574A8
S113AD8065637465640D0A0054696D6572206578A5
S113AD9070697265642028706572696F64696320E4
S113ADA073656E64696E67290D0A0000535731207C
S113ADB07075736865640D0A0000000053573220F3
S113ADC07075736865640D0A0000000053573320E2
S113ADD07075736865640D0A000000000954656DA0
S113ADE070657261747572653A202025642064650B
S113ADF0672E20430D0A000009496C6C756D696E5D
S113AE00616E63653A20202575206C780D0A000078
S113AE1009416363656C65726174696F6E3A2020E1
S113AE202575206D670D0A0053656E64696E672091
S113AE306461746120746F20534947464F58206EF3
S113AE406574776F726B2C20706C65617365207705
S113AE506169740D0A000000095365742052435A55
S113AE6031202845545349290D0A000009536574BB
S113AE702052435A322028464343290D0A00000039
S113AE80095365742052435A3320284152494229B8
S113AE900D0A0000095365742052435A3420284691
S113AEA04343290D0A000000534947464F58206484
S113AEB0657669636520697320696E20746865200E
S113AEC06E6F726D616C206D6F64650D0A00000019
S113AED0534947464F582064657669636520697312
S113AEE020696E2074686520736C656570206D6FD1
S113AEF064650D0A000000000D0A4170706C6963FE
S113AF006174696F6E2069732072656164790D0ADA
S113AF10000000002E2E2F736F757263652F6D6114
S113AF20696E2E6300000000736644727644617497
S113AF306120213D202828766F6964202A29302940
S113AF400000000025752E25752E25752E25752EDD
S113AF5025752E25752E257500000000094465769B
S113AF60696365204944203D2030780025303278DB
S113AF7020253032782000002530327820253032E8
S113AF80780D0A0009504143203D2030780000002C
S113AF90416E206572726F72206F636375727265A1
S113AFA06420696E2074686520536574566C7072F1
S113AFB04D6F64652066756E6374696F6E20282515
S113AFC064290D0A00000000416E206572726F72E0
S113AFD0206F6363757272656420696E207468659E
S113AFE0205365747570446576696365732066756E
S113AFF06E6374696F6E20282564290D0A000000B1
S113B0002D2D2D2D2D2D2D2D2D2D2D2D2D2D2D2D6C
S113B0102D2D2D2D2D2D2D2D2D2D2D2D2D2D2D2D5C
S113B0202D2D2D2D2D2D2D2D2D2D2D2D2D2D2D2D4C
S113B0302D2D2D2D2D2D2D2D2D2D2D2D0D0A446530
S113B0406D6F2070726F6A6563742C207768696312
S113B050682073656E647320646174612066726F26
S113B0606D2073656E736F72732028746865726DDA
S113B0706F6D657465722C0D0A6D61676E65746F12
S113B0806D657465722C206C696768742073656ED5
S113B090736F722920746F20534947464F58206EAE
S113B0A06574776F726B2E204D4355206F706572F7
S113B0B0617465730D0A696E20564C50522F564CBC
S113B0C05053206D6F6465732E0D0A4461746120C2
S113B0D06172652073656E7420696E2074686520E2
S113B0E0666F6C6C6F77696E672063617365733A22
S113B0F00D0A202D20557365722070726573736577
S113B1007320612070757368627574746F6E205358
S113B110573120706C61636564206F6E20746865BC
S113B120204F4C3233383520626F6172642E0D0A21
S113B13052435A31206E6574776F726B696E672063
S113B1407374616E646172642069732075736564DD
S113B15020666F72207472616E736D697373696FA8
S113B1606E2E0D0A202D205357322070757368629D
S113B1707574746F6E20707265737365642E2052DB
S113B180435A32206973207573656420666F722098
S113B1907472616E736D697373696F6E2E0D0A201C
S113B1A02D205357332070757368627574746F6EF5
S113B1B020707265737365642E2052435A3320697C
S113B1C073207573656420666F72207472616E7388
S113B1D06D697373696F6E2E0D0A202D205573658A
S113B1E072207368616B657320746865204D4355E4
S113B1F020626F6172642E2052435A342069732096
S113B2007573656420666F72207472616E736D6904
S113B2107373696F6E2E0D0A202D20506572696F4D
S113B2206469632073656E64696E672074696D6513
S113B2307220657870697265732028736574207450
S113B2406F202564207365636F6E6473290D0A2D66
S113B2502D2D2D2D2D2D2D2D2D2D2D2D2D2D2D2D1A
S113B2602D2D2D2D2D2D2D2D2D2D2D2D2D2D2D2D0A
S113B2702D2D2D2D2D2D2D2D2D2D2D2D2D2D2D2DFA
S113B2802D2D2D2D2D2D2D2D2D2D2D0D0A000000B4
S113B2904F4C323338352046572076657273696FC8
S113B2A06E3A20000D0A00002D2D2D2D2D2D2D2D53
S113B2B02D2D2D2D2D2D2D2D2D2D2D2D2D2D2D2DBA
S113B2C02D2D2D2D2D2D2D2D2D2D2D2D2D2D2D2DAA
S113B2D02D2D2D2D2D2D2D2D2D2D2D2D2D2D2D2D9A
S113B2E02D2D2D2D0D0A0000416E206572726F7296
S113B2F0206F6363757272656420696E207468657B
S113B3002053746172744170702066756E63746941
S113B3106F6E20282564290D0A0000002E2E2F644C
S113B3207269766572732F66736C5F6C70746D727C
S113B3302E6800007469636B73203E2030000000A7
S113B3402E2E2F736F757263652F73657475702E4F
S113B350630000004745545F4C50544D525F5045C4
S113B36052494F445F5449434B5328706572696F87
S113B3706453656329203C2055494E5431365F4D52
S113B380415800004745545F4C50544D525F50455E
S113B39052494F445F5449434B5328706572696F57
S113B3A06453656329203E20300000002E2E2F6454
S113B3B07269766572732F66736C5F61646331368C
S113B3C02E630000696E7374616E6365203C2041D6
S113B3D0525241595F53495A4528735F616463313E
S113B3E036426173657329004E554C4C20213D2033
S113B3F0636F6E66696700006368616E6E656C47B3
S113B400726F7570203C204144435F5343315F4366
S113B4104F554E54000000002E2E2F64726976653D
S113B42072732F66736C5F636C6F636B2E630000C3
S113B430675F7874616C304672657100675F787419
S113B440616C33324672657100000000746172678A
S113B4506574436F6E666967000000002E2E2F64CA
S113B4607269766572732F66736C5F646D612E68A2
S113B470000000006368616E6E656C203C204653DA
S113B4804C5F464541545552455F444D414D5558D6
S113B4905F4D4F44554C455F4348414E4E454C002B
S113B4A02E2E2F647269766572732F66736C5F64D7
S113B4B06D612E6300000000696E7374616E6365D4
S113B4C0203C2041525241595F53495A4528735FE9
S113B4D0646D614261736573290000006368616E85
S113B4E06E656C203C2046534C5F46454154555292
S113B4F0455F444D415F4D4F44554C455F43484182
S113B5004E4E454C00000000636F6E666967202153
S113B5103D204E554C4C000068616E646C652021E2
S113B5203D204E554C4C000073726341646472209C
S113B530213D204E554C4C00646573744164647223
S113B54020213D204E554C4C0000000028737263AE
S113B5505769647468203D3D20315529207C7C2046
S113B560287372635769647468203D3D20325529FD
S113B570207C7C20287372635769647468203D3D85
S113B58020345529000000002864657374576964E9
S113B5907468203D3D20315529207C7C2028646539
S113B5A073745769647468203D3D20325529207CAA
S113B5B07C2028646573745769647468203D3D2059
S113B5C0345529002E2E2F647269766572732F66A6
S113B5D0736C5F6770696F2E63000000696E73742B
S113B5E0616E6365203C2041525241595F53495A70
S113B5F04528735F6770696F426173657329000042
S113B600636F6E6669670000696E7374616E63656B
S113B610203C2041525241595F53495A4528735F97
S113B620666770696F426173657329002E2E2F64FB
S113B6307269766572732F66736C5F6932632E6309
S113B64000000000696E7374616E6365203C2041E4
S113B650525241595F53495A4528735F69326342D4
S113B66061736573290000006D6173746572436FC3
S113B6706E66696720262620737263436C6F636B62
S113B6805F487A006D6173746572436F6E666967B3
S113B69000000000786665720000000068616E6456
S113B6A06C65000069326348616E646C650000007B
S113B6B0736C617665436F6E66696700736C61765F
S113B6C065436F6E6669672D3E736C617665416490
S113B6D06472657373203C20736C617665436F6E8E
S113B6E06669672D3E757070657241646472657336
S113B6F0730000002E2E2F647269766572732F66B4
S113B700736C5F6C70746D722E630000696E737479
S113B710616E6365203C2041525241595F53495A3E
S113B7204528735F6C70746D724261736573290090
S113B730636F6E66696700002E2E2F6472697665EA
S113B74072732F66736C5F6C70756172742E630014
S113B750696E7374616E6365203C20415252415995
S113B7605F53495A4528735F6C7075617274426106
S113B770736573290000000068616E646C650000E5
S113B7806461746100000000636F6E6669670000A5
S113B790636F6E6669672D3E62617564526174659C
S113B7A05F427073000000006261756452617465E9
S113B7B05F4270730000000072696E6742756666CE
S113B7C06572000078666572000000007866657234
S113B7D02D3E646174610000786665722D3E64617B
S113B7E0746153697A650000636F756E74000000BC
S113B7F02E2E2F647269766572732F66736C5F7375
S113B80070692E6300000000696E7374616E636575
S113B810203C2041525241595F53495A4528735F95
S113B820737069426173657329000000636F6E660B
S113B830696720262620737263436C6F636B5F48CD
S113B8407A000000636F6E6669670000786665724F
S113B8500000000068616E646C65000068616E64DD
S113B8606C6520262620786665720000735F73700D
S113B8706948616E646C655B305D0000735F737072
S113B8806948616E646C655B315D00002E2E2F6427
S113B8907269766572732F66736C5F756172742E4C
S113B8A063000000696E7374616E6365203C2075EB
S113B8B06172744172726179436F756E7400000035
S113B8C068616E646C650000636F6E666967000092
S113B8D0636F6E6669672D3E62617564526174655B
S113B8E05F427073000000006261756452617465A8
S113B8F05F42707300000000646174610000000026
S113B90072696E6742756666657200007866657274
S113B91000000000786665722D3E646174615369AD
S113B9207A650000786665722D3E6461746100007A
S113B930636F756E740000002E2E2F647269766535
S113B94072732F66736C5F706F72742E68000000E0
S113B950636F6E6669670000AC1000004810000059
S113B96090100000760F000090100000841000007A
S113B97090100000760F00004810000048100000EE
S113B98084100000760F00006C0F00006C0F0000A4
S113B9906C0F0000D01200007C1900006A1B00002C
S113B9A06A1B00005C1900004618000046180000DD
S113B9B04E1900005C190000461800004E190000E2
S113B9C0461800005C1900004418000044180000E8
S113B9D044180000721B0000446267436F6E736F6B
S113B9E06C655F496E697400494F5F496E69740004
S113B9F04C4F475F507573680000000000F00F4023
S113BA0040F00F4080F00F40C0F00F4000F10F40B5
S113BA1053465F5061636B4672616D6500000000C0
S113BA2053465F53656E64537069446174610000EA
S113BA3053465F5265636569766553706944617402
S113BA406100000053465F5761697450696E4C652C
S113BA5076656C0053465F53656E64436F6D6D612C
S113BA606E64496E7400000053465F53746F7265D0
S113BA7044657653746174650000000053465F5357
S113BA80746F72655061796C6F61640053465F49ED
S113BA906E69740053465F47657444656661756CEE
S113BAA074436F6E6669670053465F53656E644303
S113BAB06F6D6D616E64000053465F53656E645034
S113BAC061796C6F6164000053465F54657374530D
S113BAD07069436F6E00000053465F4368616E6790
S113BAE0654E6574776F726B5374616E64617264D2
S113BAF00000000053465F53657444656661756CCD
S113BB007450415461626C650000000000F00F4005
S113BB1040F00F4080F00F40C0F00F4000F10F40A4
S113BB2053465F53657475704750494F7300000066
S113BB304D4D415F436F6E664669666F00000000BD
S113BB4041444331365F4765744368616E6E656C8A
S113BB50436F6E76657273696F6E56616C756500BE
S113BB6000F00F4040F00F4080F00F40C0F00F4055
S113BB7000F10F4000600740007007405350495FD8
S113BB80414D4C5F4D6173746572496E6974000078
S113BB905350495F414D4C5F4D6173746572476505
S113BBA07444656661756C74436F6E666967000002
S113BBB05350495F414D4C5F4D61737465724669E2
S113BBC06C6C53646B436F6E666967005350495FD6
S113BBD0414D4C5F4D617374657253656C6563745C
S113BBE044657669636500005350495F414D4C5F7D
S113BBF04D6173746572556E73656C6563744465E9
S113BC0076696365000000005350495F414D4C5F05
S113BC104D61737465725472616E7366657200006F
S113BC205072696E744669726D7761726556657299
S113BC3073696F6E0000000053657475704C505446
S113BC404D5200004C50544D525F53657454696D0D
S113BC506572506572696F64000000005365744C2E
S113BC6050544D52506572696F64416E64526573ED
S113BC706574000041444331365F476574496E730F
S113BC8074616E636500000041444331365F496E60
S113BC906974000041444331365F47657444656606
S113BCA061756C74436F6E6669670000414443318B
S113BCB0365F5365744368616E6E656C436F6E6680
S113BCC06967000041444331365F476574436861E6
S113BCD06E6E656C537461747573466C6167730042
S113BCE00670000006700000247000008E700000D2
S113BCF0247000008E7000008E7000005E700000E2
S113BD00687000008E7000008E7000008E7000005D
S113BD10727000008E7000008E7000008E70000043
S113BD208E7000007C7000007C7000008670000043
S113BD3080841E0000127A00434C4F434B5F4765DA
S113BD40744F7363304572436C6B467265710000C7
S113BD50434C4F434B5F476574457233326B436CBE
S113BD606B46726571000000434C4F434B5F47655F
S113BD70744F7574436C6B4672657100434C4F434A
S113BD804B5F5365744D63676C697465436F6E668E
S113BD9069670000444D415F48616E646C654952B7
S113BDA051000000444D415F436C6561724368611A
S113BDB06E6E656C537461747573466C6167730061
S113BDC00090044000A0044000B0044000C00440BF
S113BDD000D0044000F00F4040F00F4080F00F40CE
S113BDE0C0F00F4000F10F404750494F5F47657462
S113BDF0496E7374616E6365000000004750494FDB
S113BE005F50696E496E69740000000014001600EA
S113BE1018001A001C001E00220028001C0020002C
S113BE20240028002C003000380044003000380082
S113BE304000480050005800680080005000600036
S113BE40700080009000A000C000F000A000C000BE
S113BE50E0000001200140018001E0014001800177
S113BE60C0010002400280020003C00380020003FC
S113BE708003000480040005000680070005000616
S113BE80000700080009000A000C000F00600640CB
S113BE900070064006003410070034104932435F36
S113BEA0476574496E7374616E6365004932435F1C
S113BEB04D6173746572496E697400004932435F61
S113BEC04D617374657247657444656661756C741D
S113BED0436F6E66696700004932435F4D61737456
S113BEE065725472616E73666572426C6F636B69DE
S113BEF06E6700004C50544D525F476574496E7331
S113BF0074616E63650000004C50544D525F496E7D
S113BF10697400004C50544D525F47657444656623
S113BF2061756C74436F6E6669670000004005407C
S113BF300050054014003810150038104C5055417D
S113BF4052545F476574496E7374616E6365000093
S113BF504C50554152545F496E6974004C505541E0
S113BF6052545F47657444656661756C74436F6EC3
S113BF70666967004C50554152545F577269746545
S113BF80426C6F636B696E67000000004C50554152
S113BF9052545F52656164426C6F636B696E6700F3
S113BFA0006007400070074016003410170034107A
S113BFB05350495F476574496E7374616E636500DD
S113BFC05350495F4D6173746572496E6974000022
S113BFD05350495F4D61737465725472616E736638
S113BFE06572426C6F636B696E6700005350493031
S113BFF05F44726976657249525148616E646C653A
S113C00072000000535049315F4472697665724989
S113C010525148616E646C657200000000000000BB
S113C0200000000000C00640000000000000000006
S113C0300C003410554152545F476574496E737453
S113C040616E636500000000554152545F496E699A
S113C05074000000554152545F476574446566613D
S113C060756C74436F6E66696700000055415254E5
S113C0705F52656164426C6F636B696E67000000B8
S113C08001020000000000000000000000000100A8
S113C090504F52545F53657450696E436F6E6669B6
S113C0A06700000073717274000000004300000018
S113C0B008E0FF1FF8B5C046F8BC08BC9E467047B0
S10FC0C0F8B5C046F8BC08BC9E467047AA
S10BC0CCA443FF7F0100000002
S107C0D43904000027
S107C0D8110400004B
S113C0DC00127A00010000000000000000000000C3
S113C0EC0000000000000000000000000000000040
S113C0FC0000000000000000ACC0000000000000C4
S113C10C000000000000000000000000000000001F
S113C11C000000000000000000000000000000000F
S113C12C00000000000000000000000000000000FF
S113C13C000000000000000008E0FF1F00000000E9
S90304E90F
